S024000062696E2F6F70656E626C745F6F6C696D65785F73746D3332653430372E737265639F
S315080000000000022059020008A7020008A9020008F9
S31508000010AB020008AD020008AF02000800000000AD
S31508000020000000000000000000000000B102000807
S31508000030B302000800000000B5020008B702000875
S31508000040BB020008BD020008BF020008C102000882
S31508000050C3020008C5020008C7020008C902000852
S31508000060CB020008CD020008CF020008D102000822
S31508000070D3020008D5020008D7020008D9020008F2
S31508000080DB020008DD020008DF020008E1020008C2
S31508000090E3020008E5020008E7020008E902000892
S315080000A0EB020008ED020008EF020008F102000862
S315080000B0F3020008F5020008F7020008F902000832
S315080000C0FB020008FD020008FF0200080103000801
S315080000D003030008050300080703000809030008CE
S315080000E00B0300080D0300080F030008110300089E
S315080000F0130300081503000817030008190300086E
S315080001001B030008FD3B00081F0300082103000825
S31508000110230300082503000827030008290300080D
S315080001202B0300082D0300082F030008013C0008D4
S3150800013033030008350300083703000839030008AD
S315080001403B0300083D0300083F030008410300087D
S31508000150430300084503000847030008490300084D
S315080001604B0300084D0300084F030008510300081D
S3150800017053030008550300085703000859030008ED
S315080001805B0300085D03000810B5054C237833B9F6
S31508000190044B13B10448AFF300800123237010BD4C
S315080001A00003002000000000CCA00008084B10B592
S315080001B01BB108490848AFF300800848036803B92B
S315080001C010BD074B002BFBD0BDE81040184700BFF9
S315080001D00000000004030020CCA00008FC02002058
S315080001E000000000154B002B08BF134B9D46A3F5D6
S315080001F0803A00218B460F461348144A121A09F012
S31508000200BBFA0F4B002B00D098470E4B002B00D0A3
S3150800021098470020002104000D000D48002802D050
S315080002200C48AFF3008009F03FFA2000290000F0DF
S31508000230C5FA09F025FA00BF0000080000000220F0
S315080002400000000000000000000300202831002004
S31508000250000000000000000007498D460749084ACB
S31508000260084B9A42BEBF51F8040B42F8040BF8E754
S31508000270054880470548004700000220D8A0000826
S3150800028040000020FC0200207D2B0008E501000844
S315080002903349344A002301E041F8043B9142FBD339
S315080002A000F08CFAFEE7FEE7FEE7FEE7FEE7FEE76C
S315080002B0FEE7FEE7FEE7FEE7FEE7FEE7FEE7FEE708
S315080002C0FEE7FEE7FEE7FEE7FEE7FEE7FEE7FEE7F8
S315080002D0FEE7FEE7FEE7FEE7FEE7FEE7FEE7FEE7E8
S315080002E0FEE7FEE7FEE7FEE7FEE7FEE7FEE7FEE7D8
S315080002F0FEE7FEE7FEE7FEE7FEE7FEE7FEE7FEE7C8
S31508000300FEE7FEE7FEE7FEE7FEE7FEE7FEE7FEE7B7
S31508000310FEE7FEE7FEE7FEE7FEE7FEE7FEE7FEE7A7
S31508000320FEE7FEE7FEE7FEE7FEE7FEE7FEE7FEE797
S31508000330FEE7FEE7FEE7FEE7FEE7FEE7FEE7FEE787
S31508000340FEE7FEE7FEE7FEE7FEE7FEE7FEE7FEE777
S31508000350FEE7FEE7FEE7FEE7FEE7FEE7FEE700004C
S315080003600003002028310020704700BF704700BFF7
S31508000370704700BF08B503F06DFF08BD08B503F068
S315080003806BFF08BD08B5012003F062FF08BD00BF7A
S3150800039008B5002003F05CFF08BD00BF12230B80E0
S315080003A0004870477C00002004230B8000487047F3
S315080003B07800002010B5044C0A462146034801F08F
S315080003C061FD204610BD00BF801B0020BC970008B9
S315080003D010B5044C0A462146034801F053FD204651
S315080003E010BD00BF801B0020D097000810B5044C34
S315080003F00A462146034801F045FD204610BD00BFC8
S31508000400801B0020E097000810B5044C0A462146D8
S31508000410034801F037FD204610BD00BF801B0020B1
S31508000420F097000810B5044C0A462146034801F027
S3150800043029FD204610BD00BF801B0020F897000844
S3150800044020230B8000487047BC00002008B590F8B0
S315080004501231032B01D105F021F9002008BD00BF98
S3150800046008B505F01BF9002008BD00BF08B5084609
S3150800047005F046F9002008BD08B50B7813F0600FA3
S3150800048021D14B780A2B12D00B2B15D0062B1AD15B
S315080004904B881B0A212B05D1CA88172A28BF172281
S315080004A00A4901E00A49172201F00AFD0BE0012278
S315080004B0084901F005FD06E08B7813B9054A136073
S315080004C001E001F0BBFA002008BD00BFCE00002005
S315080004D0C50000201C03002010B50446812100F049
S315080004E00DFD0121204600F009FD002010BD00BFCA
S315080004F010B5044602234022812100F0D5FC0223D0
S3150800050040220121204600F0CFFC4023034A012166
S31508000510204600F015FD002010BD00BF401B00203E
S3150800052000487047401B0020F0B583B001210846FB
S3150800053002F060F94FF4C853009303278DF805704D
S3150800054002238DF8043000268DF806608DF80760C2
S31508000550204C6946204602F0A1F90A2208212046C5
S3150800056002F0E6F90A220B21204602F0E1F90A22F6
S315080005700C21204602F0DCF94FF4007300938DF845
S3150800058005708DF8046001258DF806508DF8076012
S315080005906946204602F082F94FF4806300938DF88D
S315080005A006508DF807508DF805706946204602F00A
S315080005B075F90A221146204602F0BAF929464FF47F
S315080005C0804002F041F92946802002F021F903B063
S315080005D0F0BD00BF00000240704700BF06E000BF44
S315080005E0013300E000231B2BF9D91046421E0028D0
S315080005F0F8D1704708B54FF47A7303FB00F0FFF79C
S31508000600EDFF08BD0C4B1968C1F3072353FA81F3B4
S31508000610C1F307421A440B0E13FA82F39BB2002267
S3150800062005E005491144087903449BB20132372A8B
S31508000630F7D9584280B270470000002008B5FFF786
S31508000640E1FF044B9B8F984201D0002008BD012092
S3150800065008BD00BF0000002008B5064B1A68064B07
S315080006609A4203D1FFF7EAFF10B908BD002008BD7A
S31508000670012008BD00000020A2E742CE08B5FFF71A
S31508000680C1FF014B988708BD0000002008B5FFF799
S31508000690E3FF68B9074A084B1A60002304E0064AD4
S315080006A01A44002111710133372BF8D9FFF7E6FFF9
S315080006B008BD00BFA2E742CE0000002038B50446B8
S315080006C00D46FFF7C9FF40B1372C08D84DB1064B88
S315080006D01C4423792B70012038BD002038BD00202A
S315080006E038BD002038BD00BF00000020F0B583B03B
S315080006F002F044FA0121084602F07CF8012400942D
S3150800070000268DF804608DF8076002258DF80550DF
S315080007106946284802F0C2F82146202002F094F8DB
S315080007202146042002F066F8234F0822062138469F
S3150800073002F0FEF808220721384602F0F9F88DF88B
S3150800074006608DF807408DF80450402300938DF815
S3150800075005506946384602F0A1F88DF80450802302
S3150800076000936946384602F099F82146284602F071
S3150800077041F8A7F5806709220521384602F0D8F81E
S3150800078009220621384602F0D3F8602300938DF833
S3150800079004508DF805508DF806608DF807406946B7
S315080007A0384602F07BF821464FF0C06002F03EF86A
S315080007B003B0F0BD000002400008024030B583B027
S315080007C0002502AC04F8015DFFF790FFFFF75EFF16
S315080007D004F080FD21462846FFF770FF9DF8073094
S315080007E0012B01D104F06AFD04F084FDFCE700BF8B
S315080007F010B50446044B1B685B6A98474FF0804364
S31508000800E2685361012010BDDC00002038B50446BB
S31508000810C3685D6815F0040F03D0044B1B689B6A18
S315080008209847E3685D60012038BD00BFDC00002002
S3150800083010B50446837A43B1D0F80C316FF34103FF
S315080008406FF30003D0F80C2113602269536823F074
S3150800085001035360054B1B689B69204698474FF078
S315080008600043E2685361012010BD00BFDC00002090
S3150800087030B583B0054600248DF8074090F812314C
S315080008808DF80730154B1B685B6998472B699A6882
S315080008904FF40064EB685C61AB7AE3B112F0010FC8
S315080008A019D095F81531012B15D19DF80730DBB213
S315080008B0032B10D1D5F80C21136843F001031360FC
S315080008C0D5F80C21136843F003031360044A13692F
S315080008D043F006031361012003B030BDDC0000209D
S315080008E000ED00E010B50446044B1B68DB6898472A
S315080008F00823E2685361012010BD00BFDC00002018
S3150800090010B50446044B1B68DB6998474FF48013FF
S31508000910E2685361012010BDDC00002010B50446D2
S31508000920044B1B681B6A98474FF40013E26853612F
S31508000930012010BDDC00002010B402691469536B55
S31508000940CB40DB01DBB22343043100EB8100826834
S31508000950906818405DF8044B704700BF2DE9F041D8
S31508000960074600F0C9FF0446002553E014F0010FBE
S315080009704ED05FFA85F84146384600F0C3FF064672
S3150800098010F0010F2BD0012605F1140307EB8303A2
S315080009905B689E60FB78B34210D105F1140307EB40
S315080009A083035B681969AA002A44D3003B44D3F839
S315080009B07C23C1F31201521AC3F88C23184B1B6807
S315080009C01B68414638469847FB78012B07D135B94D
S315080009D097F81131052B02D1384600F0A3FF16F01F
S315080009E0020F06D0022605F1140307EB83035B68A2
S315080009F09E6016F0080F0BD0094B1B689B6838469B
S31508000A009847082605F1140307EB83035B689E6085
S31508000A1001356408002CA9D10120BDE8F08100BF8A
S31508000A20DC0000202DE9F04107460D468A000A44FD
S31508000A30D3000344D3F83021D3F83411521AD3F82B
S31508000A4024319A4200D8134603F103084FEA98085E
S31508000A502B1D07EB83039B689B6927E05B1A05EB55
S31508000A608501CA003A44D2F82461B34200D81E462A
S31508000A7006F103084FEA9808AB002B44DC003C4417
S31508000A80B3B2EAB2D4F82811384600F03BFBD4F8E2
S31508000A9028313344C4F82831D4F834311E44C4F814
S31508000AA034612B1D07EB83039B689B699BB29845B2
S31508000AB00BD2AB002B44DA003A44D2F83411D2F800
S31508000AC03031994201D2002BC8D10120BDE8F0810E
S31508000AD02DE9F041074600F01FFF044600265EE0B8
S31508000AE014F0010F59D05FFA86F841463846FFF7E9
S31508000AF023FF054610F0010F1ED0012303FA06F066
S31508000B0039694A6B22EA00024A631D46321D07EB21
S31508000B10820292689360244B1B685B68414638469C
S31508000B209847FB78AB4207D136B997F81131042BB1
S31508000B3002D1384600F0F6FE15F0080F05D0082554
S31508000B40331D07EB83039B689D6015F0100F05D0D6
S31508000B501025331D07EB83039B689D6015F0400F36
S31508000B6005D04025331D07EB83039B689D6015F070
S31508000B70020F05D00225331D07EB83039B689D6092
S31508000B8015F0800F09D031463846FFF74BFF802510
S31508000B90331D07EB83039B689D6001366408002CB0
S31508000BA09ED10120BDE8F081DC0000202DE9F0414E
S31508000BB00546C268936923F010039361C3681C6AEB
S31508000BC004F00F06C4F34343022B02D0062B1CD0B5
S31508000BD02BE047F6F073234227D0C4F30A144FEAF2
S31508000BE0860808EB0603DF0007442246D7F8801379
S31508000BF000F09EFAD7F880332344C7F88033D7F835
S31508000C008C331C44C7F88C430FE0082200F2CC5101
S31508000C1000F08EFAC4F30A14B2009119CB002B44E3
S31508000C20D3F88C231444C3F88C43EA68936943F0D9
S31508000C30100393610120BDE8F08100BF2DE9F84358
S31508000C4004460025A8462F462E460269536823F017
S31508000C5001035360294600F03FFB2B460CE01A1DA2
S31508000C6004EB82029268FF21916003F1140204EBFF
S31508000C70820252689160013362789342EFD3236906
S31508000C804FF0FF329A614FF0010969F30F0569F3D6
S31508000C901F452369DD6148F00B082369C3F81480F2
S31508000CA047F00B0723691F61226913686FF30A135C
S31508000CB01360204600F036FE46F48056E3685E610F
S31508000CC0034B1B681B69204698474846BDE8F883CE
S31508000CD0DC00002038B5044600F038FCE368DD681F
S31508000CE0204600F023FC032808D10023A3704FF404
S31508000CF00073A380092363F38D2506E00123A370FF
S31508000D004023A380052363F38D25E368DD604FF454
S31508000D100053E2685361012038BD00BF2DE9F8434E
S31508000D20054600F039FB00286AD0284600F03CFB4F
S31508000D300646002868D0C0F3074818F0080F04D004
S31508000D402846FFF70BFE044600E0002418F0040FBF
S31508000D5003D02846FFF7BCFE0443F7B217F0020F8C
S31508000D6002D00223EA6853614FEA166919F0800F28
S31508000D7003D02846FFF75CFD0443C6F3072616F0A2
S31508000D80080F03D02846FFF773FD044317F0080F32
S31508000D9003D02846FFF7A6FD044317F0100F03D02B
S31508000DA02846FFF703FF044316F0100F03D0284622
S31508000DB0FFF744FF044316F0200F03D02846FFF739
S31508000DC089FF044318F0100F03D02846FFF798FD53
S31508000DD0044318F0200F03D02846FFF79FFD04436D
S31508000DE019F0400F03D02846FFF702FD044317F019
S31508000DF0040F08D02846FFF709FD2043BDE8F8830D
S31508000E000020BDE8F8832046BDE8F88338B50446D7
S31508000E1000F0A0F9012384F81231002284F8142185
S31508000E2015E091001144CB002344012183F81D11DC
S31508000E3083F81C21A3F82221002183F81F114020E2
S31508000E40C3F82401C3F82811C3F8301101326078B9
S31508000E508242E6D3002214E091001144CB002344D9
S31508000E60002183F8751383F87423A3F87A2383F88B
S31508000E7077134025C3F87C53C3F88013C3F8881347
S31508000E8001328242E8D3204600F01EFA204600F0DE
S31508000E90CBF90021204600F063FA204600F0AEFAAE
S31508000EA0204600F009FA38BD70B54DB2002D09DAB2
S31508000EB001F07F0606EB8606F40004F58C740444FC
S31508000EC0043408E001F07F0606EB8606F40004F514
S31508000ED05C740444043401F07F012170ED0F6570E1
S31508000EE0A260E37005B1E180022B01D100232371D2
S31508000EF0214600F041FB002070BD00BF10B54AB284
S31508000F00002A09DA01F07F0404EB8404E30003F500
S31508000F108C730344043308E001F07F0404EB840473
S31508000F20E30003F55C730344043301F07F01197091
S31508000F30D20F5A70194600F051FB002010BD00BFB1
S31508000F4070B501F07F04A6003519E9000D4601F5D4
S31508000F505C71014404310544C5F88023C5F888331B
S31508000F600023C5F88C3385F8753385F87443C37840
S31508000F70012B05D104EB8405EB000344C3F8842355
S31508000F8004EB8404E300034493F8743313B900F0C4
S31508000F90E7FB01E000F046FB002070BD70B501F0EC
S31508000FA07F05AE007119CC0004F58C740444211D2C
S31508000FB02E44F4000444012684F81D6184F81C516B
S31508000FC0C4F82821C4F82C210022C4F83421C4F816
S31508000FD0303115B900F0C4FB01E000F023FB002016
S31508000FE070BD00BF10B54AB2002A09DA01F07F04C5
S31508000FF004EB8404E30003F58C730344043306E02E
S3150800100001EB8104E30003F55C7303440433012414
S315080010109C7001F07F011970D20F5A70194600F0C2
S3150800102033FC002010BD00BF10B54AB2002A09DA09
S3150800103001F07F0404EB8404E30003F58C73034496
S31508001040043306E001EB8104E30003F55C73034413
S31508001050043300249C7001F07F011970D20F5A7076
S31508001060194600F02DFC204610BD00BF002361F391
S315080010700A13026911680B431360704708B50369C0
S31508001080596841F002025A600320FFF7B3FA08BD17
S31508001090C3684FF0FF325A60C3686FF080425A61E6
S315080010A0014BC268936170470008008030B583B071
S315080010B00546002401940320FFF790FAEB681A69A5
S315080010C0019201340E4A944217D8019A002AF2DA9C
S315080010D0019A42F001020192019A1A610023EA6814
S315080010E0126901920133064A934203D8019A12F013
S315080010F0010FF4D10320FFF771FA002003B030BDC9
S31508001100400D030010B4C4786CB903339B10323217
S3150800111000EB82008468002203E051F8040B20608B
S3150800112001329A42F9D300205DF8044B704700BF9C
S3150800113010B403329210D0F8D040002303E02068A0
S3150800114041F8040B01339342F9D308465DF8044B82
S31508001150704700BF30B40023C37001238370402357
S31508001160838001290DD10123C37208230370042348
S3150800117043704FF4A073C380022303724FF0A04458
S315080011800CE051B90023C3720C2303700623437085
S315080011904FF4A063C380234C00E00024C46004F528
S315080011A00063036100230FE004EB431202F51065A8
S315080011B0191D00EB81018D6002F5306203F11401FF
S315080011C000EB81014A60013342789342ECD304F57F
S315080011D08063436104F58863C0F8CC30002309E0D6
S315080011E004EB431101F5A06103F1220200EB820230
S315080011F0916001330578AB42F2D3002309E004EB92
S31508001200033101F5805103F1320200EB820291604D
S315080012100133AB42F3D304F56064C0F80C410020F7
S3150800122030BC70470000044038B50446037A012BE9
S3150800123022D10025C268936B6FF31043417A09B136
S3150800124043F480139363E268D3686FF386136FF3EE
S3150800125096536FF351436FF3D343D3602046FFF79A
S3150800126025FFE378012B19D1052363F3440545F0DF
S315080012702005E3689D6011E0C268D16841F040032B
S31508001280D360FFF713FF4FF45023627A0AB14FF485
S31508001290E813E26893631420FFF7ACF9E378012BAF
S315080012A007D1E3689D68052262F3440545F02005E9
S315080012B09D60002038BD00BFC268936843F00103F3
S315080012C093600020704700BFC268936823F001034B
S315080012D093600020704700BF00B583B000230193D8
S315080012E0019A42F020020192019A61F38A12019250
S315080012F0C26801991161C268126901920133074AED
S31508001300934203D8019A12F0200FF4D10320FFF775
S3150800131065F9002003B05DF804FB00BF400D03002B
S3150800132000B583B000230193019A42F0100201929E
S31508001330C26801991161C268126901920133074AAC
S31508001340934203D8019A12F0100FF4D10320FFF745
S3150800135045F9002003B05DF804FB00BF400D03000B
S3150800136008B5C268D3686FF35D736FF39E7301297E
S3150800137002D143F0005302E009B943F08043D36039
S315080013803220FFF737F9002008BD00BFC368586947
S3150800139000F00100704700BF08B5FFF7F7FF10F12E
S315080013A0FF3018BF012008BDC36858699B691840FB
S315080013B0704700BF0269136861F301031360704741
S315080013C038B505460024C3689C61C3686FF080423F
S315080013D05A61FFF75DFEEB7803B9102444F08044A8
S315080013E044F4701444F4605444F00C04EA689369B5
S315080013F023EA04031C439461002038BD70B50446F3
S315080014000025D0F80C311D600269136865F3CC23FA
S315080014101360C37A012B27D12E460321FFF7CAFF93
S31508001420E26880235362202262F31F4563F30F05A7
S31508001430E1688D62A02161F30F0663F31F46E36836
S31508001440C3F804614FF4907363F30F0662F31F4603
S31508001450E368C3F808614FF4A07363F30F066FF3EC
S315080014601F46E368C3F80C6110212046FFF734FFD6
S315080014702046FFF755FF236900221A6123695A613E
S3150800148023694FF0FF3199612369DA6116E0131D6C
S3150800149004EB83039B681B68002B02DA4FF090412C
S315080014A000E00021131D04EB830398680160996826
S315080014B0002008619B68FF219960013263789A428F
S315080014C0E5D3002218E002F1140304EB83035B68FA
S315080014D01B68002B02DA4FF0904100E0002102F170
S315080014E0140304EB830358680160596800200861F7
S315080014F05B68FF219960013263789A42E3D32269D7
S31508001500136943F480731361E378012B09D103232C
S31508001510402262F38A0343F4803362F35943226913
S3150800152013632046FFF74CFF002070BD03699B68D4
S31508001530C3F34103022B04D005D8012B03D00320A3
S315080015407047012070470220704700BF03699B68F7
S3150800155082691168C3F34103022B02D06FF30A01B3
S3150800156002E0032363F30A0111600269536843F436
S31508001570807353600020704730B400224B78012BEB
S3150800158008D10D782C1D00EB8404A468AB4063F3E6
S315080015900F0209E00D7805F1140400EB8404646871
S315080015A00123AB4063F31F42236813F4004F0DD1A8
S315080015B08D6865F30A03CD7865F39343C98861F3AB
S315080015C0995343F0805343F4004323600369D96970
S315080015D00A43DA61002030BC704700BF70B40022AD
S315080015E015464B78012B08D10E78311D00EB810189
S315080015F08C68B34063F30F0509E00B7803F1140414
S3150800160000EB840464680121994061F31F456FF378
S31508001610CF3222600269D36923EA0503D361002029
S3150800162070BC704738B54B78012B58D10B7804330A
S3150800163000EB83039B681A681C694B692BB96FF327
S315080016401204012363F3DC440DE063F312048D688E
S315080016502B44013BB3FBF5F363F3DC44CB78012B56
S3150800166001D163F35E740B78043300EB83039B6844
S315080016701C61C378012B07D10B78043300EB830375
S315080016809B680C695C610CE0CB78012B09D04B692F
S315080016903BB10C78012303FA04F405696B6B234309
S315080016A06B63CB78012B09D103699B6813F4807FA0
S315080016B002D142F0005201E042F0805242F0044268
S315080016C00B78043300EB83039B681A60CB78012BF5
S315080016D044D18B8A0A78C968FFF714FD3EE00B7877
S315080016E0143300EB83035B681A681C694B6933B9CA
S315080016F08B6863F31204012363F3DC440CE08D6802
S315080017002B44013BB3FBF5F3C3F3090363F3DC4452
S3150800171005FB03F363F312040B78143300EB83031E
S315080017205B681C61C378012B06D10B78143300EB78
S3150800173083035B680C695C61CB78012B06D14B7916
S3150800174013B142F0005201E042F0805242F00442E6
S315080017500B78143300EB830043681A60002038BD09
S3150800176030B482B04B78012B49D183691A681C6959
S3150800177000944C696CB99DF800406FF306048DF827
S3150800178000409DF80240012565F3C4048DF8024027
S3150800179017E08D68AC4207D94D619DF8004065F3A6
S315080017A006048DF8004005E09DF8005064F3060530
S315080017B08DF800509DF80240012565F3C4048DF8A4
S315080017C00240009C1C61C478012C06D10C780434B4
S315080017D000EB8404A4680D69656142F004421A604E
S315080017E0C378002B4CD14B69002B49D00A780123CA
S315080017F003FA02F201694B6B13434B6340E00B7823
S31508001800143300EB83035B681A681B6900934B6902
S3150800181073B98C689DF8003064F306038DF80030C0
S315080018209DF80230012464F3C4038DF802300EE0FB
S315080018308C684C619DF8003064F306038DF800301F
S315080018409DF80230012464F3C4038DF802300B7846
S31508001850143300EB83035B68009C1C61C378012B7F
S3150800186006D10B78143300EB83035B680C695C6163
S3150800187042F004420B78143300EB830043681A6085
S31508001880002002B030BC70474B78012B0DD10B7885
S31508001890043300EB830082681368002B01DA43F0F7
S315080018A0804343F40013136008E00B78143300EB0D
S315080018B083004268116841F40013136000207047E2
S315080018C04B78012B05D10B78043300EB8300806835
S315080018D004E00B78143300EB8300406802686FF36A
S315080018E05552CB78023BDBB2012B01D842F080522D
S315080018F002600020704700BF03699869DB691840D9
S31508001900000C7047143100EB81014B689A68036933
S3150800191058691040704700BF03699869DB69184029
S3150800192080B2704782B000230093C0238DF803303D
S315080019304FF00003012262F3C4038DF80230182326
S315080019408DF80030436D009A1A61C378012B08D1CF
S31508001950436D00F2CC525A61436D1A684FF08022EB
S315080019601A6002B0704700BF0346002002E001304B
S31508001970C0B201331A78002AF9D1704710B5044667
S315080019804B88012B09D1C0F81831D0F8E4359B688B
S315080019909847204600F0B4FA10BD022B29D18B884F
S315080019A013F0FF0F25D1026952681B0A013B042B6D
S315080019B017D8DFE803F003070B0F1300012363F3BF
S315080019C006120EE0022363F306120AE0032363F30A
S315080019D0061206E0042363F3061202E0052363F306
S315080019E00612044B1A60012384F81631204600F0CB
S315080019F087FA10BD801C002090F8CC350B7090F843
S31508001A00CD354B7090F8CE3590F8CF2503EB0223F1
S31508001A104B8090F8D03590F8D12503EB02238B80C4
S31508001A2090F8D23590F8D32503EB02239BB2CB80EE
S31508001A30C0F84031012380F81131704710B50446CB
S31508001A408021FFF7CFFA00212046FFF7CBFA204680
S31508001A50FFF768FF10BD00BF30B583B005460C46DA
S31508001A604A88130A013B062B67D8DFE803F00416F9
S31508001A702266665E6200D0F8EC351B680DF1060139
S31508001A8080789847E388402B03D095F81231012BCC
S31508001A9057D10823ADF8063053E0D0F8E4359B6AF1
S31508001AA00DF106018078984702234370C5F8F005C2
S31508001AB047E0D2B2052A34D8DFE802F0030B131B3D
S31508001AC0232BD0F8EC355B680DF106018078984732
S31508001AD037E0D0F8EC359B680DF106018078984719
S31508001AE02FE0D0F8EC35DB680DF1060180789847D1
S31508001AF027E0D0F8EC351B690DF106018078984788
S31508001B001FE0D0F8EC355B690DF10601807898473F
S31508001B1017E0D0F8EC359B690DF1060180789847F7
S31508001B200FE02146FFF78AFF19E02146FFF786FFF7
S31508001B3015E02146FFF782FF11E02146FFF77EFFF9
S31508001B400DE0BDF8063053B1E28842B19A4228BF8B
S31508001B501A46ADF806200146284600F0B1F903B04A
S31508001B6030BD00BF38B504468B88E3B9CB88D3B9F6
S31508001B708D7805F07F0590F81231032B02D1FFF717
S31508001B805DFF38BD80F814512946FFF76FFA2046E5
S31508001B9000F0B6F91DB1022384F8123138BD0123CD
S31508001BA084F8123138BD2046FFF748FF38BD00BF1C
S31508001BB010B504468B78214A1370012B02D9FFF71A
S31508001BC03DFF10BD90F81221022A02D0032A10D038
S31508001BD030E05BB180F81031032280F812211946F3
S31508001BE000F0F4FA204600F08BF910BD00F088F9F1
S31508001BF010BD5BB9022280F8122180F8103119460F
S31508001C0000F0F0FA204600F07BF910BD90F81011AC
S31508001C108B420CD000F0E6FA084B197884F81011BC
S31508001C20204600F0D3FA204600F06AF910BD00F00D
S31508001C3067F910BDFFF702FF10BD00BF240300209F
S31508001C4008B5CB88012B02D0FFF7F8FE08BD90F83F
S31508001C501231022B02D0032B05D00AE001220649D5
S31508001C6000F02EF908BD012200F5887100F028F968
S31508001C7008BDFFF7E3FE08BD2C03002008B590F861
S31508001C801231023B012B0DD80122084B1A60D0F8FD
S31508001C90183113B10322054B1A600222034900F0DA
S31508001CA00FF908BDFFF7CAFE08BD00BF20030020D4
S31508001CB010B5044690F81231023B012B0DD84B881B
S31508001CC0012B0CD10023C0F81831D0F8E4359B68F5
S31508001CD09847204600F014F910BDFFF7AFFE10BD77
S31508001CE008B54B78092B1BD8DFE803F011171A142F
S31508001CF01A08051A0E0BFFF7AFFE13E0FFF732FFBF
S31508001D0010E0FFF755FF0DE0FFF79AFF0AE0FFF72F
S31508001D10B5FF07E0FFF732FE04E0FFF7C9FF01E071
S31508001D20FFF78CFE002008BD38B504460D4690F82E
S31508001D301231032B0FD10B79012B09D8D0F8E435D2
S31508001D409B689847EB8843B9204600F0D9F804E029
S31508001D50FFF774FE01E0FFF771FE002038BD00BFF3
S31508001D6038B505460C468A88D1B26378012B27D048
S31508001D70002B49D0032B40F0818090F81231022BBA
S31508001D8002D0032B07D017E0002977D0802975D019
S31508001D90FFF728F972E0638823B919B1802901D0C1
S31508001DA0FFF720F9D5F8E4359B6821462846984779
S31508001DB0284600F0A5F861E02146FFF73FFE5DE002
S31508001DC090F81231022B02D0032B07D018E0002915
S31508001DD054D0802952D0FFF705F94FE06388002BCD
S31508001DE04CD149B1802907D0FFF71EF9D5F8E4355B
S31508001DF09B68214628469847284600F081F83DE02A
S31508001E002146FFF71BFE39E090F81231022B02D06B
S31508001E10032B06D02FE089B380292FD0FFF7E2F8ED
S31508001E202CE052B2002A10DA01F07F0101EB8101A1
S31508001E30CB00034493F81E311BB10122104B1A60E4
S31508001E4013E000220E4B1A600FE0002A0DDB01EBAF
S31508001E508101CB00034493F876331BB10122084B6A
S31508001E601A6002E00022064B1A600222044928463C
S31508001E7000F026F802E02146FFF7E0FD002038BD15
S31508001E8028030020D0B170B50D4616460446FFF764
S31508001E906BFD0130400080B23080287003236B70E0
S31508001EA0022307E05A1CD2B20134E9540233DBB2EA
S31508001EB00021A95421780029F4D170BD704700BFCC
S31508001EC010B504461346C4F83C21C4F8382102224A
S31508001ED080F811210A460021FFF760F8002010BD9E
S31508001EE008B513460A460021FFF758F8002008BD32
S31508001EF008B513460A460021FFF722F8002008BD58
S31508001F0010B50446042380F8113100231A461946F1
S31508001F10FFF744F82046FFF705FD002010BD00BF77
S31508001F2010B50446052380F8113100231A461946D0
S31508001F30FFF706F82046FFF7F5FC002010BD00BFA6
S31508001F400369024A12685A6000207047801C002004
S31508001F5010B50446D0F8E8351B699847032384F87A
S31508001F601231002010BD00BF08B590F8123180F874
S31508001F701331042380F81231D0F8E835DB68984726
S31508001F80002008BD08B5D0F8E435DB6903B19847E9
S31508001F90002008BD08B5D0F8E4351B6A984700202C
S31508001FA008BD00BF08B5D0F8E4355B6A984700203D
S31508001FB008BD00BF10B50446D0F8E8355B699847F8
S31508001FC0012384F81531002010BD00BF10B5044662
S31508001FD0D0F8E8359B699847D4F8E4355B68002162
S31508001FE020469847002084F8150110BD10B5044610
S31508001FF0002340221946FEF757FF0023402280217E
S315080020002046FEF751FF012384F81231D4F8E8354B
S315080020105B68A0789847002010BD00BF10B582B055
S3150800202004466946FFF7E8FC9DF8001001F01F0317
S31508002030012B08D013B1022B0AD00EE069462046C0
S31508002040FFF74EFE0EE069462046FFF76DFE09E0F3
S3150800205069462046FFF784FE04E001F08001204629
S31508002060FEF7C0FF002002B010BD00BF10B5044641
S31508002070002947D190F81131022B38D1D0F83821F0
S31508002080D0F824319A4211D9D21AC0F83821C17829
S31508002090012904D1D0F828110B44C0F8283192B28E
S315080020A0D4F828112046FFF71BFF20E0D0F83C1192
S315080020B0B1FBF3F203FB121262B98B420AD8D0F8CD
S315080020C04031994206D21146FFF70AFF0023C4F8A9
S315080020D040310CE0D4F8E435DB682BB194F81221D2
S315080020E0032A01D1204698472046FFF719FF94F89E
S315080020F01631012B11D12046FFF722FF002384F861
S3150800210016310AE00A46D0F8E4355B692BB190F837
S315080021101211032901D111469847002010BD00BFAE
S3150800212010B5044659BB90F81131032B32D1D0F8BB
S315080021309033D0F87C23934214D99B1AC0F8903375
S31508002140C178012904D1D0F880131144C0F880134E
S315080021509A4228BF1A4692B2D4F880132046FFF74F
S31508002160C7FE17E0D0F8E4351B6923B190F81221B1
S31508002170032A00D198472046FFF7C2FE0AE00A461E
S31508002180D0F8E4359B692BB190F81211032901D1D7
S3150800219011469847002010BDF8B504460D46164668
S315080021A01F46FEF7C1F9C4F8E475069BC4F8E8357E
S315080021B0C4F8EC6529462046FEF728FED4F8E8352B
S315080021C01B6898472046FEF707FAF8BD10B504467F
S315080021D0D0F8E4351B689847D4F8E8359B689847E3
S315080021E0002010BD08B5D0F8E4355B689847002094
S315080021F008BD00BF0A4B0B4A9A6000221A60DB60D2
S315080022005A6040225A719A884FF4C86161F30C02E9
S315080022109A808022DA7041F20C0203498B5070478B
S31508002220001D0020101D002000800240054B064AB4
S315080022309A60DB6000221A605A6041F21002034974
S315080022408B507047002A002050230020008002404F
S315080022502DE9F041B2B001214FF0F05000F0CAFA72
S315080022600121472000F0C6FA01214FF4804000F012
S31508002270EBFA012000F0C4F98E23309300258DF87F
S31508002280C65002248DF8C4408DF8C7508DF8C54055
S315080022905B4F30A9384600F001FB0B220121384676
S315080022A000F046FB0B222146384600F041FB0B2284
S315080022B00321384600F03CFB0B220721384600F084
S315080022C037FB4FF4006330938DF8C6508DF8C44041
S315080022D08DF8C7508DF8C54007F5C05730A9384660
S315080022E000F0DCFA0B221146384600F021FB3223B7
S315080022F030938DF8C6508DF8C4408DF8C7508DF8C8
S31508002300C540DFF80C8130A9404600F0C7FA0B2219
S315080023100121404600F00CFB0B220421404600F048
S3150800232007FB0B220521404600F002FB4FF4C04391
S3150800233030938DF8C6508DF8C4408DF8C7508DF887
S31508002340C54030A9384600F0A9FA0B220D213846B7
S3150800235000F0EEFA0B220E21384600F0E9FA01F0F9
S3150800236005FD01F01FFF01F025FF0128FBD001A89C
S3150800237001F008FD0025019508954FF400730B93AD
S315080023800C954FF000430F9320231293149515953F
S3150800239016954FF4006309934FF48043069313E0B0
S315080023A0ACB20221204601F03DFD60F31F46032131
S315080023B0204601F037FD60F30F06124B9E4205D00A
S315080023C0114B9E4202D001351F2DE9D9202D04D983
S315080023D04FF4A1710D4802F0E5FFA9B201A801F07A
S315080023E07FFD20B940F24711084802F0DBFFFFF7EE
S315080023F01DFFFFF7FFFE01F01BFF32B0BDE8F081BD
S315080024000000024019162200F1C0070010980008C3
S3150800241000080240064B08221A7000225A7027222A
S315080024209A706922DA705B221A7145225A717047CE
S315080024309C1A002008230370002343702723837007
S315080024406923C3705B23037145234371704700BF3B
S3150800245038B50D4BDB7813F0800F13D10A4D688819
S31508002460C0F30D0422460949094807F07AF9EB78C2
S3150800247043F08003EB70012141F20803054AD1506D
S31508002480204638BD002038BD001D0020101D002044
S31508002490A42A00200080024038B50F4BDB7813F0E1
S315080024A0800FFAD10D4B1C880D4D22460D49284642
S315080024B007F057F9084B9D6000221A6010219970A1
S315080024C05A60C4F30B049C80B022DA70012141F2F1
S315080024D00403054AD15038BD002A0020102A0020DE
S315080024E050230020A42A00200080024008B503F0EB
S315080024F02BFA08BD30B585B004460D46038A9BB253
S3150800250023F44053CA881343038283899BB223F476
S31508002510B05323F00C01A8882A896B890243134318
S315080025200B43A381A38A9BB223F44073AA8913435E
S31508002530A382684600F002F9204B9C4203D003F5BB
S3150800254080639C4201D1039A00E0029AA38913F49E
S31508002550004F08D002EB820202EB8202296849008A
S31508002560B2FBF1F107E002EB820202EB8202296874
S315080025708900B2FBF1F1124BA3FB01235B091B0196
S315080025801A09642000FB1212A18911F4004F08D021
S31508002590D20032320A49A1FB0212C2F342121A438E
S315080025A007E0120132320649A1FB0212C2F34312B6
S315080025B01A4392B2228105B030BD00BF0010014017
S315080025C01F85EB5129B183899BB243F4005383815C
S315080025D0704783899BB223F400539BB2838170476B
S315080025E0C1F30801818070478088C0F308007047EE
S315080025F00388194201D0012070470020704700BFA8
S31508002600014B1860704700BFDC00274208B501215E
S315080026104FF4006000F034F900214FF4006000F038
S315080026202FF908BD10B40B4C636823F4FD4121F063
S315080026307F01027D83681A4343681A43C3681A43B5
S3150800264003681343026913430B4363605DF8044B45
S31508002650704700BF002C0140014B1860704700BF4F
S31508002660A0802542014B1860704700BF002C01402E
S31508002670024B186800F00300704700BF002C0140A9
S3150800268010B40368094CA360E36823F4FF6121F0E2
S315080026900701426883681A43C368134302691343F0
S315080026A00B43E3605DF8044B704700BF002C014004
S315080026B0014B1869C0B27047002C014082B0002354
S315080026C00193034B03440193019B186802B07047BA
S315080026D0142C014010B4036809494B6243688B62A5
S315080026E0CB6A23F0F7048268C3681A430369134365
S315080026F0426913432343CB625DF8044B704700BF1E
S31508002700002C0140014BD3F880007047002C014093
S31508002710014BC3F880007047002C0140034B5B6BEC
S31508002720034201D00120704700207047002C014069
S31508002730014B9863704700BF002C014010B4294B29
S315080027409B6803F00C03042B05D0082B06D053BB5B
S31508002750254B036029E0254B036026E0214B5A6888
S315080027605B6803F03F0312F4800F09D01F4AB2FBDF
S31508002770F3F21C4B5B68C3F3881303FB02F208E011
S31508002780194AB2FBF3F3174A5168C1F3881101FBE2
S3150800279003F2144B5B68C3F3014301335B00B2FBDE
S315080027A0F3F3036001E0104B03600E4CA368C3F318
S315080027B003130F49CB5CDAB20368D3404360A268BF
S315080027C0C2F382228A5CD2B223FA02F28260A2683B
S315080027D0C2F342328A5CD2B2D340C3605DF8044B7E
S315080027E0704700BF003802400024F400001BB70001
S315080027F00C01002021B1054B1A6B10431863704772
S31508002800024A136B23EA000010637047003802403F
S3150800281021B1054B5A6B104358637047024A536BF4
S3150800282023EA0000506370470038024021B1054B87
S315080028301A6C104318647047024A136C23EA0000A6
S31508002840106470470038024021B1054B5A6C10439A
S3150800285058647047024A536C23EA00005064704774
S315080028600038024021B1054B1A69104318617047B8
S31508002870024A136923EA00001061704700380240D3
S3150800288021B1054B5A6A104358627047024A536A87
S3150800289023EA0000506270470038024070B40023F3
S315080028A03AE001229A400C68A24334D104685D00DC
S315080028B00322AA40D2431440046006680C79AC404F
S315080028C0344304600C79013CE4B2012C15D88468C1
S315080028D02240826084684A79AA4022438260466818
S315080028E09AB20124944026EA0404446046688C7926
S315080028F004FA02F292B232434260C4689AB25600AF
S315080029000322B24024EA0202C260C668CC7904FAFD
S3150800291005F23243C26001330F2BC2D970BC70472F
S315080029200369194201D0012070470020704700BF93
S3150800293030B401F007039B009A40C908083150F8E3
S3150800294021400F2505FA03F324EA030340F8213052
S3150800295050F821301A4340F8212030BC704700BF98
S31508002960054B1B69002B05DA034B044A5A6002F132
S3150800297088325A60704700BF003C02402301674511
S31508002980024A136943F0004313617047003C024052
S31508002990014BD860704700BF003C02400E4BDB6815
S315080029A013F4803F10D10C4BDB6813F0100F0DD1D8
S315080029B0094BDB6813F0EF0F0AD1074BDB6813F0FE
S315080029C0020F07D00720704701207047052070477F
S315080029D00620704708207047003C024000B583B0C7
S315080029E008238DF80730FFF7D9FF8DF8070003E0B5
S315080029F0FFF7D4FF8DF807009DF80730DBB2012BEF
S31508002A00F6D09DF8070003B05DF804FB70B50546DF
S31508002A1031B1012906D0022907D14FF4007606E024
S31508002A20002604E04FF4807601E04FF44076FFF785
S31508002A30D5FF08281ED1104C236923F4407323615F
S31508002A4023691E432661236923F0F803236123695A
S31508002A501D4345F002052561236943F4803323614C
S31508002A60FFF7BCFF236923F002032361236923F0E0
S31508002A70F803236170BD00BF003C024070B50546EF
S31508002A800E46FFF7ABFF082813D10A4C236923F437
S31508002A9040732361236943F400732361236943F078
S31508002AA0010323612E60FFF799FF236923F00103D1
S31508002AB0236170BD003C024082B00023019300935D
S31508002AC02A4A136843F480331360284B1B6803F4BF
S31508002AD000330093019B01330193009B1BB9019BB3
S31508002AE0B3F5A06FF1D1214B1B6813F4003F02D058
S31508002AF00123009301E000230093009B012B32D1B0
S31508002B001A4B1A6C42F080521A6419490A6842F440
S31508002B1040420A609A689A609A6842F400429A604B
S31508002B209A6842F4A0529A60124A5A601A6842F0A9
S31508002B3080721A600D4B1B6813F0007FFAD040F2C2
S31508002B4005620D4B1A60A3F580639A6822F00302AA
S31508002B509A609A6842F002029A60044B9B6803F0F6
S31508002B600C03082BF9D102B0704700BF00380240A9
S31508002B70007000400C544007003C024010B5104C51
S31508002B80D4F8883043F47003C4F888300D4B1A68BB
S31508002B9042F001021A60002199601A6822F08472D4
S31508002BA022F480321A60084A5A601A6822F480228F
S31508002BB01A60D960FFF780FF4FF00063A36010BD6D
S31508002BC000ED00E00038024010300024FEE700BFA8
S31508002BD02DE9F04182B001210C20FFF70BFE2C4CA9
S31508002BE00C2208212046FFF7A3FE0C2209212046C5
S31508002BF0FFF79EFE0C220A212046FFF799FE0C22BB
S31508002C000B212046FFF794FE0C2211462046FFF7BB
S31508002C108FFE204F0C2202213846FFF789FE4FF41B
S31508002C207063009301258DF805504FF002088DF862
S31508002C30048000268DF806608DF807506946204600
S31508002C40FFF72CFE0423009369463846FFF726FE55
S31508002C504FF4805300938DF8076069462046FFF7C6
S31508002C601DFE4FF4006700978DF804808DF8076005
S31508002C7069462046FFF712FE29463846FFF7E4FD67
S31508002C8029464FF48000FFF7B5FD02B0BDE8F08194
S31508002C9000080240000C024010B54FF4803400E0F2
S31508002CA0013C24B18020FFF739FD0028F8D02CB16B
S31508002CB040F2FF50FFF73CFD002010BD032010BD79
S31508002CC008B5104B5A6B4FF4803302E0013B0D4AAE
S31508002CD0526B12F0450F01D1002BF7D113B112F048
S31508002CE0040F04D00420FFF723FD032008BD12F0CB
S31508002CF0400F04D04020FFF71BFD002008BD002030
S31508002D0008BD00BF002C014008B50B4B5B6B01E00A
S31508002D10094B5B6B13F0450FFAD013F0040F04D080
S31508002D200420FFF705FD032008BD40F2FF50FFF71A
S31508002D30FFFC002008BD00BF002C014008B50F4B62
S31508002D405B6B01E00D4B5B6B13F0450FFAD013F08C
S31508002D50040F04D00420FFF7EBFC032008BD13F092
S31508002D60010F04D00120FFF7E3FC012008BD40F263
S31508002D70FF50FFF7DDFC002008BD00BF002C014016
S31508002D8010B50446444B5B6B01E0434B5B6B13F099
S31508002D90450FFAD013F0040F04D00420FFF7C8FC3F
S31508002DA0032010BD13F0010F04D00120FFF7C0FC6B
S31508002DB0012010BDFFF77CFCA04243D140F2FF5032
S31508002DC0FFF7B6FC0020FFF779FC344B0340DBB372
S31508002DD000283BDB10F0804F3AD110F0005F39D164
S31508002DE010F0805F38D110F0006F37D110F0806F87
S31508002DF036D110F0807F35D110F4000F34D110F49D
S31508002E00800F33D110F4001F32D110F4801F31D156
S31508002E1010F4002F30D110F4802F2FD110F4003F7A
S31508002E202ED110F4803F2DD110F4004F2CD110F480
S31508002E30804F2BD110F4005F2AD110F0080F29D04B
S31508002E401A2010BD102010BD002010BD1C2010BD7A
S31508002E50092010BD0A2010BD0B2010BD0C2010BD86
S31508002E600D2010BD0E2010BD0F2010BD102010BD66
S31508002E70112010BD122010BD132010BD142010BD46
S31508002E80152010BD162010BD172010BD182010BD26
S31508002E90192010BD002010BD002C014008E0FFFDE0
S31508002EA038B504460D461E4B5B6B01E01C4B5B6B4D
S31508002EB013F0450FFAD013F0040F04D00420FFF7DF
S31508002EC037FC032038BD13F0010F04D00120FFF7AB
S31508002ED02FFC012038BDFFF7EBFBA04218D140F2CA
S31508002EE0FF50FFF725FC0020FFF7E8FB10F4604FC2
S31508002EF003D1000C2880002038BD10F4005F09D1EA
S31508002F0010F4804F08D110F4004F07D00F2038BDB9
S31508002F10102038BD132038BD102038BD002038BD1C
S31508002F20002C0140F0B583B00E46002300930193B0
S31508002F305648082202601024446040228260C3601A
S31508002F404FF480630361FFF79BFB2046FFF718FFEA
S31508002F50002840F094804E4B1B68A3404B48036002
S31508002F6037244460402383600023C3604FF48063A2
S31508002F700361FFF785FB2046FFF702FF00287FD194
S31508002F8044484FF0FF3303600823436030238360CF
S31508002F900223C3600024046101234361FFF79AFBFF
S31508002FA03A4804603325456040238360C4604FF483
S31508002FB080630361FFF764FB2846FFF7E1FE0546D9
S31508002FC000285ED127460EE04FF40010FFF7A6FB57
S31508002FD020B1FFF797FB4DF827000137013442F27D
S31508002FE010739C424ED82C4B5A6B40F22A631A42F5
S31508002FF0EAD00820FFF792FB20B10820FFF798FBDC
S31508003000042040E00220FFF789FB20B10220FFF7E9
S315080030108FFB022037E02020FFF780FB20B120201D
S31508003020FFF786FB06202EE04FF40070FFF776FBCD
S3150800303028B14FF40070FFF77BFB072023E040F22E
S31508003040FF50FFF775FB00990B0203F47F0343EA71
S3150800305001630A0A02F47F42134343EA1163736069
S3150800306001990B0203F47F0343EA01630A0A02F497
S315080030707F42134343EA11633360284603E002E0C4
S3150800308001E000E0042003B0F0BD00BFE803002023
S315080030908C03002034030020002C014010B582B0B8
S315080030A00446002000900190FFF708FB10F0007F0F
S315080030B05CD16946324B1888FFF734FF002857D190
S315080030C0012C2AD1019B13F4802F52D02C4B1B685C
S315080030D01B042C4803603724446040238360002384
S315080030E0C3604FF480630361FFF7CAFA2046FFF70F
S315080030F047FE00283FD12348022303600624446084
S31508003100402383600023C3604FF480630361FFF7A5
S31508003110B7FA2046FFF734FE30E0019B13F4803FF0
S315080031202AD0174B1B681B041648036037244460D3
S31508003130402383600023C3604FF480630361FFF775
S315080031409FFA2046FFF71CFEC0B90E48002303600D
S315080031500624446040228260C3604FF480630361A2
S31508003160FFF78EFA2046FFF70BFE07E00E2005E074
S3150800317004E0252002E001E02520FFE702B010BDAB
S315080031808C030020E803002000B583B001238DF8E6
S3150800319007304FF400610648FFF7C2FB10B9002359
S315080031A08DF807309DF8070003B05DF804FB00BFF3
S315080031B00008024070B582B000248DF807406648C2
S315080031C076230375046044608460C4600461FFF775
S315080031D029FA0320FFF746FA0120FFF73DFA5F4870
S315080031E0046044608460C4604FF480630361FFF741
S315080031F047FAFFF751FD8DF807009DF8073013F0E1
S31508003200FF0F03D09DF80700C0B2A3E053484FF460
S31508003210D573036008234360402383600023C3609B
S315080032204FF480630361FFF72BFAFFF749FD8DF82A
S3150800323007009DF8073013F0FF0F05D10122484B10
S315080032401A604FF0804611E044480026066037248D
S31508003250446040238360C6604FF480630361FFF7D0
S315080032600FFA2046FFF78CFD8DF807003B48002330
S3150800327003603724446040228260C3604FF4806351
S315080032800361FFF7FDF92046FFF77AFD8DF8070081
S315080032909DF8073013F0FF0F40D058E02F48002361
S315080032A003603725456040228260C3604FF480631F
S315080032B00361FFF7E5F92846FFF762FD8DF8070079
S315080032C09DF8073013F0FF0F03D09DF80700C0B232
S315080032D040E046F0004343F4801320480360292366
S315080032E04360402383600023C3604FF48063036117
S315080032F0FFF7C6F9FFF708FD8DF807009DF80730B8
S3150800330013F0FF0F03D09DF80700C0B222E000209B
S31508003310FFF7D4F90246C00F013402E00020044644
S31508003320024618B94FF6FE739C42B7D94FF6FE739C
S315080033309C4206D91B238DF807309DF80700C0B2BA
S3150800334008E012F0804F02D00222054B1A609DF861
S315080033500700C0B202B070BD74030020E803002065
S315080033605C03002010B582B00123ADF80630FFF7E4
S315080033707FF900286AD0394B1B68042B20D03848BF
S315080033800023036002224260C0228260C3604FF4B9
S3150800339080630361FFF774F9FFF7D0FC002857D163
S315080033A0FFF78CF92F4C20600420FFF787F960603F
S315080033B00820FFF783F9A0600C20FFF77FF9E0608B
S315080033C0264B1B68012B03D9062B01D0022B12D1E1
S315080033D02348002303600324446040228260C360BC
S315080033E04FF480630361FFF74BF90DF106012046A0
S315080033F0FFF756FD68BB194B1B68042B2AD0BDF88E
S315080034000630194A13601B041548036009234360F4
S31508003410C02383600023C3604FF480630361FFF712
S315080034202FF9FFF78BFCB8B9FFF748F90F4C206066
S315080034300420FFF743F960600820FFF73FF9A06012
S315080034400C20FFF73BF9E060002005E0252003E0AB
S3150800345002E001E00020FFE702B010BD5C03002097
S31508003460E8030020600300208C0300204C030020A2
S31508003470F0B40346A44A146880F85640A34A128852
S31508003480A0F85420A24D2A68100EC1B28E091E70EB
S31508003490C0F38300587001F003019970C2F3074125
S315080034A0D970C2F307211971D2B25A7169680A0E26
S315080034B01201DA80C1F30740DA8892B242EA1012A2
S315080034C0DA8000F00F001872080AC2B2D5095D72D8
S315080034D0C0F380159D72C0F34015DD72C0F3001568
S315080034E01D7300255D73012C44D8800200F44060EA
S315080034F018611A69890001F47F7111431961844AB8
S315080035009268100EC1B21C6944EA91141C61C0F39A
S31508003510C200187501F007015975110CC1F3421064
S315080035209875C1F38200D875490001F0060119762D
S31508003530C2F30722197E41EAD21119761C690134B1
S315080035409C64DD64187E0230012505FA00F0C71771
S31508003550A0FB040104FB0711C3E912011C7AE4B2BB
S3150800356005FA04F41C65A4FB006704FB0177C3E9AC
S31508003570126721E0022C1FD1090401F47C1119619C
S31508003580634A9268100E196941EA0021196119699E
S31508003590C2F3074001431961C2F3072218690021E3
S315080035A0013041F10001C90441EA5031C004986470
S315080035B0D9644FF400711965C2F380115976520027
S315080035C002F07E029A765248027A997E41EAD21130
S315080035D0997602F07F02DA76C1680A0ED009187762
S315080035E0C2F341105877C2F382009877920002F02E
S315080035F00C02DA77080CC2B2DC7F44EA9214DC7754
S31508003600C0F3401083F82000002083F8210002F060
S31508003610010283F822200A0AD4B2E50983F8235066
S31508003620C2F3801583F82450C2F3401583F8255059
S31508003630C2F3001583F82650C2F3810283F82720C7
S3150800364004F0030483F82840C1F3460183F82910DF
S31508003650012483F82A402F4D2A68110E83F82C106E
S31508003660C2F307410902D985C2F30726D98D89B263
S315080036703143D98512061A636A68160E196B41EA30
S3150800368006411963110C1E6B090201F47F4131438F
S315080036901963196BC2F3072631431963D2B283F84B
S315080036A03420AA68110E83F83510110C090699639F
S315080036B0110A9E6B090401F47F0131439963996BE2
S315080036C0120202F47F420A439A63EA68996B41EA56
S315080036D012619963110C93F83C60C1F303153543E5
S315080036E083F83C50090201F47061D987C2F30725B3
S315080036F0D98F89B22943D987C2F3460283F8402075
S3150800370083F84140F0BC70475C0300208C0300201E
S315080037104C030020600300201C4B1B68032B2CD095
S31508003720022B2CD8B0F5805F2BD010B5B0F5006F02
S3150800373012D10120FFF7B2FC044620BB144800232F
S3150800374003750360436083604FF40062C2600361DF
S31508003750FEF768FF204610BD0020FFF79FFC0446D1
S3150800376090B90B4800230375036043608360C36008
S315080037700361FEF757FF204610BD2720704700203B
S3150800378070472720704710BD10BD00BF5C0300209E
S315080037907403002010B5094B186007245C604022AA
S315080037A09A600022DA604FF480621A611846FEF7C2
S315080037B067FF2046FFF7E4FA10BD00BFE8030020C4
S315080037C000B583B000238DF80730FFF701FAFEF73E
S315080037D01DFFFFF7EFFC8DF807009DF8073013F083
S315080037E0FF0F03D09DF80700C0B237E0FFF7BAFD18
S315080037F08DF807009DF8073013F0FF0F03D09DF8EA
S315080038000700C0B22AE01748002303750360436027
S315080038108360C3600361FEF705FF1348FFF728FEC0
S315080038208DF807009DF8073013F0FF0F08D10E4BEF
S31508003830B3F8540000040021FFF7ACFF8DF8070029
S315080038409DF8073013F0FF0F05D14FF40060FFF71E
S3150800385063FF8DF807009DF80700C0B203B05DF856
S3150800386004FB00BF7403002090030020F8B505464A
S315080038701646BDF8181000225248027052480260D7
S31508003880524802605248C262524A1268022A04D159
S31508003890720A42EAC3564FF400710F464E48016059
S315080038A010234360402383600023C3604FF4806382
S315080038B00361FEF7E5FE4FF4803400E0013C24B1D5
S315080038C08020FEF72BFF0028F8D01020FFF758FAC3
S315080038D0002874D141484FF0FF33036047609023B6
S315080038E083600223C3600027076101234361FEF753
S315080038F0F1FE394806601124446040238360C7609E
S315080039004FF480630361FEF7BBFE2046FFF738FAE3
S31508003910064680B154E04FF40040FEF7FFFE50B172
S3150800392005E0FEF7EFFE45F82400013400E0002428
S31508003930072CF6D92035264B5A6B40F22A631A42D1
S31508003940E9D00820FEF7EAFE20B10820FEF7F0FECF
S315080039500420F8BD0220FEF7E1FE20B10220FEF7A2
S31508003960E7FE0220F8BD2020FEF7D8FE20B1202071
S31508003970FEF7DEFE0620F8BD4FF40070FEF7CEFE19
S3150800398058B14FF40070FEF7D3FE0720F8BDFEF7D6
S31508003990B9FE45F8040B013C01E04FF0FF344FF443
S315080039A00010FEF7BBFE08B1002CF0D140F2FF5024
S315080039B0FEF7BEFE00220A4B1A603046F8BDF8BD77
S315080039C0F8BD00BF3003002070030020FC03002070
S315080039D0002C01405C030020E8030020340300208B
S315080039E01C0100202DE9F04105461646BDF81810C1
S315080039F000225648027056480260564802605648E9
S31508003A00C262564A1268022A04D1720A42EAC356A8
S31508003A104FF400710F465248016010244460402359
S31508003A2083600023C3604FF480630361FEF728FEBA
S31508003A302046FFF7A5F9002840F08380484806602D
S31508003A4018244460402383600023C3604FF48063D6
S31508003A500361FEF715FE2046FFF792F90446002893
S31508003A6071D140484FF0FF3303604760902383606D
S31508003A700026C660066101234361FEF72BFE2AE095
S31508003A804FF48040FEF74AFE28B3C6F50078B8F131
S31508003A901F0F1BD8734213F0030F02D14FEA980881
S31508003AA003E04FEA980808F10108002705E055F8F1
S31508003AB0040BFEF72DFE013704364745F7D30AE017
S31508003AC055F82700FEF724FE013700E00027072FE8
S31508003AD0F6D920352036204B5A6B40F21A631A4223
S31508003AE0CED00820FEF71AFE28B10820FEF720FEE1
S31508003AF00420BDE8F0810220FEF710FE28B102205E
S31508003B00FEF716FE0220BDE8F0811020FEF706FE3D
S31508003B1028B11020FEF70CFE0520BDE8F0814FF411
S31508003B200070FEF7FBFD30B14FF40070FEF700FEA3
S31508003B300720BDE8F08100220B4B1A602046BDE83D
S31508003B40F081BDE8F081BDE8F08100BF30030020B8
S31508003B5070030020FC030020002C01405C030020B9
S31508003B60E8030020340300201C010020D8B138B532
S31508003B7005460E4B1B681B040D4803600D24446064
S31508003B80402383600023C3604FF480630361FEF71C
S31508003B9077FD2046FFF7F4F8044630B9FEF78EFDA8
S31508003BA02860204638BD2620704738BD8C03002083
S31508003BB0E803002000B583B000230193FFF7E4FA79
S31508003BC0012807D101A8FFF7D1FF28B90198C0F34A
S31508003BD0432002E0FF2000E0FF2003B05DF804FB6D
S31508003BE008B5FFF7E7FF042803D0FF2803D1022012
S31508003BF008BD002008BD012008BD00BF704700BFF2
S31508003C00704700BF00B597B0FFF7DAFD48B9084A14
S31508003C10137803F0FE0313706846FFF729FC0020AB
S31508003C2003E00122024B1A70032017B05DF804FB6B
S31508003C302001002008B50122064B1A7038B9FFF793
S31508003C40CFFF20B9034A137803F0FE031370014B24
S31508003C50187808BD2001002070B5ADF5027D0E4626
S31508003C601546B8B11BE062194FF40073009352026F
S31508003C70002302A8FFF7FAFD98B9FFF7B1FF01285C
S31508003C80FBD04FF4007202A906EB442005F069FD4B
S31508003C90234644B15C1E002BE5D1012004E0012037
S31508003CA002E0012000E000200DF5027D70BD00BF96
S31508003CB0F0B5ADF5037D0F461646C0B11CE04FF4CE
S31508003CC000752A4607EB442102A805F04AFDA21909
S31508003CD000955202002302A8FFF784FE08B10528C2
S31508003CE00CD1FFF77DFF0128FBD0234644B15C1EAB
S31508003CF0002BE4D1012004E0012002E0012000E0CD
S31508003D0000200DF5037DF0BD174B1B7813F0010F4E
S31508003D101FD103291FD8DFE801F002041318002079
S31508003D207047D0B910B596B014466846FFF7A0FBA1
S31508003D30129B5B0A139A43EAC2532360002010E0E1
S31508003D404FF4007313800020704740B92023136096
S31508003D5070470320704704207047002070470020F2
S31508003D60704716B010BD00BF2001002008B501211C
S31508003D704FF00070FEF776FD00214FF00070FEF759
S31508003D8071FD08BD0023036043608360C36003615F
S31508003D9043618361C361036243628362C3620363EF
S31508003DA043638363C36340220264202242648364BC
S31508003DB0C364036543658365C365036680224266FB
S31508003DC08366C366036743678367C3674FF080628A
S31508003DD0C0F880204FF00072C0F884204FF0807140
S31508003DE0C0F888104FF40011C0F88C10C0F8903055
S31508003DF0C0F89430C0F89830C0F89C30C0F8A030AD
S31508003E00C0F8A420C0F8A8304FF40032C0F8AC209F
S31508003E104FF48072C0F8B020C0F8B430C0F8B8309B
S31508003E20704700BF82B000230193124A136903F05A
S31508003E301C03C00280B20343890101F4F8610B43F5
S31508003E4043F001031361019B01330193094B1B697D
S31508003E5013F0010F03D0019A074B9A42F3D9019A3E
S31508003E60064B9A4203D0034B586980B200E0002003
S31508003E7002B0704700800240FEFF0400FFFF040006
S31508003E8010B483B000230193124C236903F01C037A
S31508003E90C00280B20343890101F4F8610B4343F081
S31508003EA0030362612361019B01330193094B1B697B
S31508003EB013F0010F03D0019A074B9A42F3D9019ADE
S31508003EC0064B9A4201D1002000E0012003B05DF8BC
S31508003ED0044B704700800240FEFF0400FFFF040009
S31508003EE070B586B004460D46002305930093924BA1
S31508003EF01E6926F01C0601A8FEF720FC029A8F4BC5
S31508003F0013448F498B4202D846F008060EE08D4BC3
S31508003F1013448D498B4202D846F00C0606E08B4BBB
S31508003F2013448B4A934201D946F00406824B1E611C
S31508003F304FF4004200212846FFF7A2FF0646002854
S31508003F4000F0F7804FF08063059302E0059B013B84
S31508003F500593059E002EF9D12368002B4CD0009BB3
S31508003F600133009301212846FFF75CFF00F00400A7
S31508003F7080B218B9009A774B9A42F0D9009A764BD4
S31508003F809A4200F0D680002100914FF480522846CC
S31508003F90FFF776FF002800F0CB80009B01330093E3
S31508003FA001212846FFF73EFF00F0200080B218B92D
S31508003FB0009A684B9A42F0D9009A674B9A4200F0E9
S31508003FC0B8800023009310212846FFF72BFF00F046
S31508003FD004039BB21BB14FF40063236201E0002384
S31508003FE0236200F002039BB213B1002363611CE055
S31508003FF04FF48043636118E0226AC2F3CF02636913
S31508004000C3F34F031A4300212846FFF739FF064634
S31508004010002800F08E806FF07F43059302E0059B31
S31508004020013B0593059B002BF9D1434B1A684B4975
S3150800403011406068A2681043E26810432269104381
S3150800404062691043A2691043E2691043226A104369
S31508004050626A1043A26A1043E26A1043226B104355
S31508004060626B02430A431A60A16BE26B1143226C2E
S315080040701143626C1143A26C1143E26C1143226D29
S315080040801143626D0A435A60A26D9A60E26DDA6066
S315080040909A694FF641711140206E626E42EA0040FD
S315080040A0A26E1043E26E1043226F1043626F024302
S315080040B00A439A61A16FE26F0A43DA6141F2180571
S315080040C05A5927491140D4F88000D4F8842010435F
S315080040D0D4F888201043D4F88C201043D4F89020C4
S315080040E01043D4F894201043D4F898201043D4F8F9
S315080040F09C201043D4F8A02002430A435A51D4F80E
S31508004100A410D4F8A8201143D4F8AC201143D4F84D
S31508004110B0200A43D4F8B41042EA8101D4F8B82092
S315080041200A4342F4000203F580531A60012600E0B0
S315080041300646304606B070BD0080024000D3CEFE6B
S31508004140BFE1E40040F1E9FD3F787D0100796CFCB0
S31508004150005A6202FEFF0400FFFF04000F8120FFE1
S31508004160233FDEF828B1064A136843F008031360B4
S315080041707047034A136823F008031360704700BFAB
S315080041800080024028B1064A136843F0040313600E
S315080041907047034A136823F004031360704700BF8F
S315080041A000800240024A136843F001031360704717
S315080041B000900240044B1B6813F0010F01D0012048
S315080041C070470020704700BF00900240034941F243
S315080041D018028B5843F480138B50704700800240B6
S315080041E038B1084941F218028B5843F400538B50F2
S315080041F07047044941F218028B5823F400538B5038
S31508004200704700BF0080024038B1084941F21802E1
S315080042108B5843F002038B507047044941F2180249
S315080042208B5823F002038B50704700BF0080024072
S3150800423008B50120FFF796FFFFF7C8FF0120FFF733
S31508004240A1FF0120FFF7CCFF0120FFF7DDFF08BD26
S31508004250704700BF704700BF704700BF08B501210F
S315080042600448FEF75DFB012801D1002008BD0120A6
S3150800427008BD00BF0000024000B5C7B04FF48C72FD
S315080042800021684605F078FA69460A4803F0E8FC12
S3150800429038B9009B3BB19DF8083013F0100F04D0D5
S315080042A004E0002002E0002000E0012047B05DF8AD
S315080042B004FB00BF249800080048704724980008AB
S315080042C008B50748002380F828320A22054903F072
S315080042D049F918B90122024B83F8282208BD00BF04
S315080042E0000400204498000810B50D4B93F82832B6
S315080042F0012B02D10A4803F0EDFB01F025FB00F182
S31508004300640403E001F020FB844205D340210548FC
S31508004310FEF76EF90028F5D0034803F0C7FC10BD78
S3150800432000040020001401402498000808B5044B36
S3150800433093F82832012B02D1014803F0CBFB08BDC4
S315080043400004002010B504460F4B93F82832012BC1
S3150800435015D10D4903F032FD002810DA0A4800236A
S3150800436080F8283203F0B6FB09E00848FEF738F96A
S3150800437080210648FEF73CF90028F9D00134217857
S315080043800029F2D110BD00BF00040020001401402E
S315080043900022014B5A7070472C060020034BFE2260
S315080043A0DA7018710222A3F8442070472C06002000
S315080043B010B5054C00232370FFF7EAFFFF23E370CF
S315080043C00123A4F8443010BD2C060020064BFF221A
S315080043D0DA7000221A71597859719A71DA711A725B
S315080043E00622A3F8442070472C06002008B50020B2
S315080043F0FFF7D4FF08BD00BF084BFF22DA70084A52
S315080044009A6400221A715A719A710721D9711A721F
S315080044105A729A720822A3F8442070472C06002084
S3150800442054980008044BFF22DA7042689A64012205
S31508004430A3F84420704700BF2C06002008B5312099
S31508004440FFF7ACFF08BD00BF38B5084CFF23E37083
S3150800445000252571657100F011FFA071E5712572BF
S3150800446065720723A4F8443038BD00BF2C06002027
S3150800447038B500F065FB18B91020FFF78FFF38BD77
S31508004480FFF786FF0D4C01252570FF23E3701023E7
S3150800449023710023637100F0F1FEA07100F0FCFEA9
S315080044A0E07100F0F9FEC0F3072020726572A5726C
S315080044B00823A4F8443001F04FFA38BD2C06002032
S315080044C038B50546447800F0D9FE0138844203DD44
S315080044D02220FFF763FF38BD084C6A78A16C201DBF
S315080044E001F05AFCFF23E3706B78A26C1344A364B3
S315080044F06B780133A4F8443038BD00BF2C06002081
S3150800450038B50446457800F0B9FE0138854203DD22
S315080045102220FFF743FF38BD6168084DA964627819
S31508004520281D01F039FCFF23EB706378AA6C13444D
S31508004530AB6463780133A5F8443038BD2C060020F7
S31508004540F8B505461746002406E015F8013B1C4455
S31508004550E4B200F00DFE31464E1E0029F5D13C604E
S315080045600120F8BD10B5084CFF23E370E21D416831
S31508004570A06CFFF7E5FF207100236371A371082380
S31508004580A4F8443010BD00BF2C06002038B50546F7
S315080045900D4B9C6C00F072FE6A1C411E204601F011
S315080045A0DFF918B93120FFF7F9FE38BD064CFF23AD
S315080045B0E37000F063FE0138A36C1844A06401237D
S315080045C0A4F8443038BD00BF2C06002038B5044690
S315080045D0457800F053FE0238854203DD2220FFF7B6
S315080045E0DDFE38BD0F4BFF22DA700122A3F8442006
S315080045F0617831B901F0C4F990B93120FFF7CEFEE0
S3150800460038BDA21C074B986C01F0AAF918B93120DD
S31508004610FFF7C4FE38BD6378024A916C0B44936475
S3150800462038BD00BF2C06002008B54168074B986CBA
S3150800463001F09AF918B93120FFF7B0FE08BD034B0F
S31508004640FF22DA700122A3F8442008BD2C060020B8
S3150800465008B501F07DFB034BFF22DA700122A3F8AF
S31508004660442008BD2C06002008B589B200F0E0FDFC
S3150800467008BD00BF054B00221A709A6483F84320D0
S31508004680A3F844209A705A70704700BF2C06002081
S31508004690024B187800B10120704700BF2C06002095
S315080046A00022024B83F84320704700BF2C060020E7
S315080046B008B50378FF2B02D1FFF7DAFE50E0334A3C
S315080046C01278012A60D1C93B352B46D8DFE803F0BA
S315080046D03345454245453F363C39454545454545BB
S315080046E0454545454545454545454545454545456C
S315080046F045454545454545454545241E1B214545F2
S315080047004527452A2D30FFF7DBFE29E0FFF7F8FE9F
S3150800471026E0FFF787FE23E0FFF724FF20E0FFF7F8
S315080047206BFE1DE0FFF762FE1AE0FFF74FFE17E08B
S31508004730FFF73EFE14E0FFF729FF11E0FFF746FFFB
S315080047400EE0FFF781FE0BE0FFF76EFF08E0FFF7CC
S315080047507FFF05E0FFF772FE02E02020FFF71EFE4E
S315080047600A4B93F84330012B02D11020FFF716FEAF
S31508004770064BB3F94410002906DD1846012380F8D4
S3150800478043300330FFF770FF08BD00BF2C0600203A
S3150800479010B5FDF75DFE48B3384A1080384B9C8942
S315080047A04FF4006003F058FC84420DD1012003F059
S315080047B08DFC324B1B88CBB104F00CFCFDF76CFE6C
S315080047C000222E4B1A8011E02D4B9C8940F60600DC
S315080047D003F042FC844209D104F08CFB274B1B886A
S315080047E023B1FDF759FE0022244B1A8001F0ACF8DC
S315080047F0244B1B68984232D303F5FA73214A136097
S31508004800002413E0204A682303FB04231F4A13608D
S31508004810022003F05BFC194B1B8833B104F0DAFB6A
S31508004820FDF73AFE0022154B1A800134002CE9D018
S31508004830002412E0164B03EB8413164A1360052076
S3150800484003F044FC0D4B1B8833B104F0C3FBFDF7A2
S3150800485023FE0022094B1A800134002CEAD001F00D
S3150800486073F80D4B1B68984206D303F51C53103397
S31508004870094A136004F00CFB10BD00BF102A002083
S31508004880A42A0020880600202C2A0020282A002096
S31508004890E8300020202A00207C0600201F4B1B78C9
S315080048A0002B39D110B5FDF7D3FC01F04DF800F512
S315080048B0FA701B4B186001F047F800F51C501030D1
S315080048C0184B186003F06EFB174A002313805380B9
S315080048D0164A13805380164A138053804EF60300F7
S315080048E003F0A0FBFDF796FD124C2046FDF7A2FD4E
S315080048F00621204604F056FD04F072FD00F032FD54
S3150800490042F20F73984203D842F2107000F024FD69
S315080049100122094B1A7010BD704700BF2101002003
S31508004920880600207C060020A02A00209C2A002059
S31508004930982A0020800600207806002008B5002264
S31508004940034B1A70034B1B780BB9FFF7A7FF08BD7B
S31508004950210100207806002038B50F4B1B78012B63
S3150800496019D10E4B1D68EB692B62002306E01A1D50
S31508004970C45C2A4482F8204001339BB28AB293422F
S31508004980F5D3111DA5F8641005F1200004F0E8F927
S31508004990EB690133EB6138BD78060020282A002030
S315080049A008B5044B1B78012B01D1FFF7F1FE002057
S315080049B008BD00BF7806002010B5194B1C68194BB6
S315080049C01B7813F0400F05D00123E3610023A4F8F8
S315080049D0643010BD13F0010F02D00022A4F8642041
S315080049E013F0040F06D0B4F8641019B104F12000CE
S315080049F004F0B6F90B4B1B7813F0020F0ED00A4BD6
S31508004A0019880B1F402B09DC0023A4F86430074BD8
S31508004A1018680439C9B20430FFF74AFE10BD00BF52
S31508004A20282A00201C2A0020102A0020242A0020D8
S31508004A30034601310D4AA2FB0323DB08F9D110B462
S31508004A4000230B70094BA3FB0023DB081A4603EB74
S31508004A5083035C00031B303301F8013D1046002A2E
S31508004A60F0D108465DF8044B704700BFCDCCCCCCDE
S31508004A7000F00F03092802D903F13700704710B573
S31508004A8003F1300404F042FE2044437803F00303A4
S31508004A90022B00D1203CE0B210BD00BF38B5054658
S31508004AA00C460009FFF7E4FF207005F00F00FFF73A
S31508004AB0DFFF60700023A370204638BDF8B50746AF
S31508004AC0002634461EE0BD5D04F020FE28444378E7
S31508004AD003F00303022B00D1203DEBB2A3F1300211
S31508004AE0D2B2162A12D8A3F13A01C9B206290FD9A9
S31508004AF0092A01D9373BDAB22301DBB21344DCB207
S31508004B000136F6B2012EDED92046F8BD0020F8BDE2
S31508004B100020F8BD08B50022054B1A70054906485D
S31508004B2002F0F4FC18B17721044800F03BFC08BDFC
S31508004B30CC0600205C980008D8060020609800087B
S31508004B40034B1B780BB9012070470020704700BF44
S31508004B50CC06002008B500F0ADFB01280AD0084BAA
S31508004B601B784BB9FFF788FB012807D10122044BB4
S31508004B701A7008BD002008BD002008BD002008BD29
S31508004B80CC06002038B50546047804F0BFFD20445D
S31508004B90437803F00303022B00D1203C532C0FD19A
S31508004BA004F0B4FD6B781844427812F0040F09D06B
S31508004BB0312B09D0322B09D0332B09D1022038BD2D
S31508004BC0032038BD032038BD002038BD012038BD7C
S31508004BD0032038BD70B506460230FFF76FFF05465D
S31508004BE084B204363046FFF769FF2844C5B2013C53
S31508004BF0A4B20236012CF5D8ED43EDB23046FFF7E4
S31508004C005DFF854201D0002070BD012070BD00BF48
S31508004C10F8B5044616460F4601B120B940F261219F
S31508004C204D4800F0BFFB2046FFF7ACFF05460328BA
S31508004C3000F08A802046FFF7CDFF002800F0868026
S31508004C40012D25D015B1022D4CD082E0A01CFFF70E
S31508004C5035FF85B2201DFFF731FF00023860A01D21
S31508004C60FFF72CFF3B68184438600834E81E05B285
S31508004C704EB92846F8BD2046FFF720FFF055023406
S31508004C800137BFB200E00027AF42F4DB2846F8BD83
S31508004C90A01CFFF713FF85B2201DFFF70FFF0004C6
S31508004CA03860A01DFFF70AFF3B6803EB0020386059
S31508004CB004F10800FFF702FF3B68184438600A341D
S31508004CC0281F05B24EB92846F8BD2046FFF7F6FE5E
S31508004CD0F05502340137BFB200E00027AF42F4DBDB
S31508004CE02846F8BDA01CFFF7E9FE85B2201DFFF790
S31508004CF0E5FE00063860A01DFFF7E0FE3B6803EB03
S31508004D000040386004F10800FFF7D8FE3B6803EB63
S31508004D100020386004F10A00FFF7D0FE3B6818440B
S31508004D2038600C34681F05B24EB92846F8BD2046CF
S31508004D30FFF7C4FEF05502340137BFB200E0002782
S31508004D40AF42F4DB2846F8BD0020F8BD4FF0FF302F
S31508004D50F8BD0020F8BD00BF6098000870B5AC4BE0
S31508004D601B78002B00F0E781012B29D100F0F4FD18
S31508004D70FFF7A6FAA748FFF7E5FAA748FFF7E2FA0A
S31508004D80FFF79AFA01220146A44802F0EBFB30B17C
S31508004D90A348FFF7D7FA0120FFF7C8FA70BDA14864
S31508004DA0FFF7D0FAA048FFF7CDFAA048FFF7CAFAEE
S31508004DB09F4B00221A605A600222954B1A7070BDEA
S31508004DC0022B40F0EF809B4C04F50C724FF4807177
S31508004DD0994802F0C9FF94F841326BB19048FFF741
S31508004DE0B1FA0220FFF7A2FA04F50C7002F072FE7F
S31508004DF00022874B1A7070BDB0B18F48002200F5AB
S31508004E00C071FFF705FF0446B0F1FF3F0DD1844896
S31508004E10FFF798FA0320FFF789FA804802F05AFE4E
S31508004E2000227B4B1A7070BD0024002C5BDD804B82
S31508004E305B6833B9804BD3F880217D4B1A605C6080
S31508004E4051E07D4AD2F88011794A12681A44914293
S31508004E5003D12344764A536045E07248FFF772FA55
S31508004E607648FFF76FFA764E714D31466868FFF758
S31508004E70DFFD3046FFF766FA7248FFF763FA3146F8
S31508004E80E878FFF70BFEB11CA878FFF707FE311D7F
S31508004E906878FFF703FEB11D2878FFF7FFFD304657
S31508004EA0FFF750FA6848FFF74DFA6968286800F076
S31508004EB05BFD60B95A48FFF745FA0520FFF736FA51
S31508004EC0564802F007FE0022514B1A7070BD55482D
S31508004ED0FFF738FA5548FFF735FA574BD3F88021CC
S31508004EE0534B1A605C60534BD3F84422D3F83C32D8
S31508004EF09A4240F020810021484802F0FDFD60B149
S31508004F004748FFF71FFA0420FFF710FA434802F054
S31508004F10E1FD00223E4B1A7070BD454B5B68002BC5
S31508004F2039D04048FFF70EFA4448FFF70BFA444DCC
S31508004F303F4C29466068FFF77BFD2846FFF702FAD3
S31508004F404048FFF7FFF92946E078FFF7A7FDA91CB7
S31508004F50A078FFF7A3FD291D6078FFF79FFDA91D1F
S31508004F602078FFF79BFD2846FFF7ECF93648FFF750
S31508004F70E9F96168206800F0F7FC60B92848FFF78E
S31508004F80E1F90520FFF7D2F9244802F0A3FD002233
S31508004F901F4B1A7070BD2348FFF7D4F903221C4B28
S31508004FA01A7070BD032B40F0C680224C04F50C72B3
S31508004FB04FF48071204802F0D7FE94F841326BB165
S31508004FC02248FFF7BFF90220FFF7B0F904F50C7085
S31508004FD002F080FD00220E4B1A7070BD002839D0F1
S31508004FE0154800F5807200F5C071FFF711FE0546F9
S31508004FF0B0F1FF3F2FD11648FFF7A4F90320FFF7BA
S3150800500095F9064802F066FD0022014B1A7070BD3C
S31508005010CC060020789800089C980008080900200B
S31508005020C4980008CC980008D4980008F898000896
S31508005030D0060020D8060020300B0020289900084A
S315080050408C06002034990008D89900085099000861
S31508005050749900080025002D40DD3748FFF772F9DE
S31508005060364C21462846FFF7E3FC2046FFF76AF947
S315080050703348FFF767F9334E214696F88301FFF761
S315080050800DFDA11C96F88201FFF708FD211D96F873
S315080050908101FFF703FDA11D96F88001FFF7FEFCCD
S315080050A02046FFF74FF92848FFF74CF906F58072B6
S315080050B02946D6F8800100F053FC60B92348FFF76B
S315080050C041F90620FFF732F9214802F003FD0022D4
S315080050D0204B1A7070BD2048FFF734F91F4BD3F8E0
S315080050E04422D3F83C329A4225D11D48FFF72AF9C3
S315080050F000F046FC60B91548FFF724F90720FFF7CA
S3150800510015F9134802F0E6FC0022124B1A7070BD1E
S315080051101148FFF717F91348FFF714F90C4802F07E
S31508005120D9FC1148FFF70EF900220A4B1A70FFF74F
S31508005130DBF800F00DFE70BD989900088C0600207B
S31508005140A8990008300B0020D8990008C4980008D0
S3150800515008090020CC060020CC980008D8060020B4
S31508005160C0990008DC990008F4990008704700BF48
S31508005170704700BF10B5FFF77DFA00F049FE064CF0
S315080051800123237000F01EFB0023237000F0D2F9E0
S315080051900223237010BD00BF2201002000B583B092
S315080051A00DF107011E4800F03FFF012807D1012233
S315080051B01C4B1A709DF807101948FFF779FA0DF17C
S315080051C00701174800F044FB012807D10022154BB8
S315080051D01A709DF807101248FFF76AFA0DF10701D1
S315080051E00F4800F013FA012807D102220D4B1A7056
S315080051F09DF807100A48FFF75BFA0DF10701084802
S31508005200FFF7CEFB012807D10322064B1A709DF83B
S3150800521007100348FFF74CFA03B05DF804FB00BF1C
S31508005220B40C00202201002008B500F0BDF908BD25
S3150800523038B504460D46104B1B78012B02D1C9B26E
S3150800524000F0A0FE0C4B1B781BB9E9B2204600F013
S31508005250D7FA094B1B78022B03D1E9B2204600F096
S31508005260ADF9054B1B78032B03D1E9B22046FFF7AE
S3150800527073FBFFF715FA38BD22010020054B1B7892
S31508005280012B05D0022B01D0402070473F207047E4
S315080052900820704722010020054B1B78012B05D0FA
S315080052A0022B01D0402070473F20704708207047E6
S315080052B02201002008B5FFF7EBF908BD08B5FFF78E
S315080052C03DFB0322024B1A7000F052F808BD00BFDE
S315080052D02201002008B500F037FDFFF747FF00F070
S315080052E011FB00F039FBFFF715FCFFF743FF00F051
S315080052F04DF808BD08B5FFF73BFF00F017FBFFF7B1
S315080053002DFDFFF74BFF00F001F808BD08B5FFF7C4
S31508005310D1FF012819D0FFF713FCB0B10B4B1B784E
S31508005320012B12D100F010FB094B1A68094B1B68B8
S31508005330134403F5FA73984207D30022034B1A70F5
S31508005340FFF708FC08B900F003FD08BDF80C0020BB
S31508005350F40C0020FC0C0020014B1860704700BFBD
S31508005360F40C0020014B1868704700BFF40C0020AD
S3150800537008B5044B1B78012B03D100F0E5FA024B64
S31508005380186008BDF80C0020FC0C002008B50122A6
S31508005390034B1A70FFF7ECFFFFF7B8FF08BD00BF15
S315080053A0F80C002008B5FFF7E3FEFCE7094B03F10C
S315080053B01801002205E09A74596118331831013230
S315080053C0D2B2002AF7D09A7400225A61014A024BD7
S315080053D01A607047880D0020840D00200B4B1B684F
S315080053E073B110B45C69094A146019749860D8607E
S315080053F000225A741860013908445860987C01E004
S31508005400FF2070475DF8044B704700BF840D0020ED
S3150800541038B504460D46012804D940F2B711154897
S31508005420FFF7C0FF62002244D300134A13445A7C94
S315080054301B7C9A421AD062002244D3000E4A1344B7
S31508005440DA6815705A7C01325A74DA680132DA6001
S315080054505B689A420CD9084A63001819C1000846C5
S31508005460515803461344D960012038BD002038BD81
S31508005470012038BD209A0008880D002008B501468D
S31508005480024B1878FFF7C4FF08BD00BFFC0D0020CB
S3150800549038B504460D46012804D940F2D9111448F6
S315080054A0FFF780FF04EB4402D300124A1344587CEA
S315080054B0E0B162002244D3000E4A13449A68127877
S315080054C02A705A7C013A5A749A6801329A605B6863
S315080054D09A420AD9074A63001819C1000846515862
S315080054E0034613449960012038BD012038BD00BF2A
S315080054F0209A0008880D002008B50146024B187846
S31508005500FFF7C6FF08BD00BFB80D002010B504465A
S31508005510012804D940F2F9110448FFF743FF04EBC8
S315080055204404E300024A1344587C10BD209A00083C
S31508005530880D002030B583B0FFF738FF134C4021A3
S31508005540601CFFF74BFF2070114D4021681CFFF7C8
S3150800555045FF28702378FF2B01D0FF2803D18A2125
S315080055600C48FFF71FFF0C4B00930C4B0C4A01210C
S315080055700C48FCF711FEFFF7F5FEB0F5FA6F03D2FB
S315080055804FF4FA60FFF7E8FE03B030BDFC0D0020CB
S31508005590B80D0020209A0008400000209000002046
S315080055A05C000020400E002008B50348FBF766FDA6
S315080055B00020FEF74DFE08BD400E002070B50646D9
S315080055C00D463F2903D9B4210F48FFF7EBFE2846BD
S315080055D0FFF754FF012803D0B8210B48FFF7E2FE76
S315080055E000240CE0FFF7C4FD305DFFF747FF0128F4
S315080055F003D0C1210448FFF7D5FE0134A4B2ABB2EB
S315080056009C42EFD370BD00BF209A000870B50646CD
S315080056100D461D48FBF782FB1C4B1C788CB91C48B1
S31508005620FFF76AFF01282DD1194B1B78013BDBB226
S315080056303E2B27D80122154B1A700022154B1A70DB
S3150800564020E0144B1B78013311481844FFF754FF28
S315080056500446012813D10F4B1A780132D2B21A70B8
S315080056600B4B1B789A420CD10B49304600F094FB41
S315080056700022064B1A70074B1B782B7002E0002499
S3150800568000E00024204670BD400E0020F90D0020E1
S31508005690000D0020400D0020010D002030B583B01C
S315080056A0134B1878FFF732FF00B30546402800D998
S315080056B04025002412E00DF107010D4B1878FFF77D
S315080056C0E7FE012804D040F241110A48FFF76AFEB6
S315080056D09DF80720084B1A550134E4B2A542EAD8CA
S315080056E02B46054A81210548FBF758FC03B030BD17
S315080056F0FC0D0020209A0008440D0020400E0020D2
S3150800570070B500EB8000C300104A1344B3F88C63ED
S31508005710002410E00E4B1D78FAF702FF015D2846BB
S31508005720FFF776FE012804D04FF4B0710948FFF759
S3150800573039FE0134A4B2B442ECD3FAF7F1FE4023A1
S31508005740024601210148FBF7FBFB70BD400E002015
S31508005750B80D0020209A000810B5044680210F488D
S31508005760FCF746FFB0B121460C48FCF739FF00F0BC
S31508005770EBF800F10A0405E0FFF7FAFC00F0E4F89C
S31508005780844209D380210548FCF732FF0028F3D06C
S31508005790012010BD002010BD002010BD00140140DE
S315080057A010B5044620210648FCF722FF012805D13A
S315080057B00348FCF719FF2070012010BD002010BD1A
S315080057C00014014010B584B04FF4614300930023E0
S315080057D0ADF80430ADF80630ADF80830ADF80C3049
S315080057E00C23ADF80A30054C69462046FCF782FEC4
S315080057F001212046FCF7E6FE04B010BD0014014066
S3150800580070B506460D46402903D979210F48FFF79A
S31508005810C9FD2846FFF7A0FF012803D07D210B48C4
S31508005820FFF7C0FD00240CE0FFF7A2FC305DFFF790
S3150800583093FF012803D086210448FFF7B3FD0134FE
S31508005840A4B2ABB29C42EFD370BD00BF489A000821
S3150800585070B5244B1C78ACB92348FFF7A1FF012883
S315080058603ED1214B1B78013BDBB23F2B38D800F0E9
S315080058706BF81E4B186000221D4B1A700122194B3B
S315080058801A702DE006460D46194B1B78013316484B
S315080058901844FFF785FF0446012813D1144B1A78DC
S315080058A00132D2B21A70104B1B789A4215D111499F
S315080058B0304600F071FA00220A4B1A700C4B1B781E
S315080058C02B700DE000F040F8084B1B6864339842D3
S315080058D005D90024034B1C7002E0002400E00024D4
S315080058E0204670BD76140020341400207814002059
S315080058F075140020351400200022014B1A607047E9
S3150800590010E000E008B5FFF7F7FF054B054A5A60B7
S3150800591000229A6005211960034B1A6008BD00BF72
S3150800592010E000E03F9002007C140020044B1B6846
S3150800593013F4803F03D0034A13680133136070479A
S3150800594010E000E07C14002008B5FFF7EFFF014BDC
S31508005950186808BD7C14002008B500F01FF908BDBA
S3150800596008B500F027F908BD08B500F059F908BDD3
S3150800597008B500F09DF908BD08B500F0E1F908BDC5
S3150800598008B500F06DF9034610B100F0B9F9034601
S31508005990184608BD38B50546002419E0FFF7E8FBA8
S315080059A004EB440293000C4AD358AB420ED804EBDE
S315080059B044018A0008490A44526813449D4205D2A4
S315080059C004EB440083000B44187A38BD0134E4B272
S315080059D0082CE3D9FF2038BDA09A000808B5C1F302
S315080059E0080353B90368994209D040F8041B4FF4D9
S315080059F0007200F0D1F9012008BD002008BD012081
S31508005A0008BD00BF2DE9F04107460068FFF7C2FF51
S31508005A10FF282ED0FCF7A4FFF320FCF7B9FFFCF70C
S31508005A20BDFF012818D1FCF7ABFF0020BDE8F081C7
S31508005A303E68A30006EB03083B445D68FFF798FB46
S31508005A4029464046FDF71AF808280AD156F82430A0
S31508005A509D4208D1013400E000247F2CE8D90124B6
S31508005A6002E0002400E00024FCF78AFF2046BDE897
S31508005A70F0810020BDE8F08138B50D460B4B984201
S31508005A8007D004460A4B994205D0FFF7BBFF18B961
S31508005A9008E0084C00E0054C29462046FFF79EFF23
S31508005AA010B938BD002038BD204638BD8014002006
S31508005AB000C00008841600202DE9F04106460C4671
S31508005AC017461D4621F4FF7828F001080368B3F14C
S31508005AD0FF3F04D14146FFF781FF034630B33368E1
S31508005AE0984505D041463046FFF7C6FF0646D0B171
S31508005AF03368E41A34440434FFF73AFB331DE31AD7
S31508005B00B3F5007F07D308F500713046FFF7B4FFF9
S31508005B10064650B1041D17F8013B04F8013B013D48
S31508005B20EAD1012302E0002300E000231846BDE87D
S31508005B30F08100BF884229D838B504460D460228A8
S31508005B4026D90B2926D8FCF70BFFF320FCF720FFF4
S31508005B50FCF724FF012813D1FCF712FF002038BDFB
S31508005B60FFF706FB02210C4B33F81400FCF74EFF37
S31508005B70082803D0FCF704FF002038BD0134E4B23E
S31508005B80AC42EDD9FCF7FCFE012038BD0020704779
S31508005B90002038BD002038BD709A00084FF0FF334A
S31508005BA0024A1360024A1360704700BF8416002039
S31508005BB08014002070B54B1E154C241AA34221D818
S31508005BC016460D460446FFF7E5FEFF281CD02819A1
S31508005BD00138FFF7DFFEFF2818D024F4FF7323F0FF
S31508005BE001030C4A934206D12B46324621460A48FF
S31508005BF0FFF762FF70BD2B46324621460748FFF77E
S31508005C005BFF70BD002070BD002070BD002070BD18
S31508005C10FFFF0F0800C0000880140020841600202B
S31508005C204A1E0E4B1B1A9A4212D870B50D460446E8
S31508005C30FFF7B0FE064628190138FFF7ABFEFF2E20
S31508005C4008D0FF2808D001463046FFF773FF70BD1D
S31508005C5000207047002070BD002070BDFFFF0F08B0
S31508005C60114B1B68B3F1FF3F18D000B583B00E4B3C
S31508005C7059689A681144DA6811441A6911445A69CC
S31508005C8011449A691144DA698B185B4202AA42F8F0
S31508005C90043D04210548FFF78DFF01E00120704708
S31508005CA003B05DF804FB00BF8014002088C100081B
S31508005CB00D4B1A6804331B6813440C4A12681344C4
S31508005CC00B4A126813440B4A11680B4404321268D3
S31508005CD01A44094B1B681344084A1268D34201D177
S31508005CE0012070470020704700C0000808C000085F
S31508005CF00CC0000810C0000818C0000888C10008B9
S31508005D0008B50D4B1B68B3F1FF3F04D00A48FFF7EF
S31508005D1079FE034668B1094B1B68B3F1FF3F05D00E
S31508005D200648FFF76FFE034610B902E0012300E0BC
S31508005D300123184608BD00BF8014002084160020E1
S31508005D400048704700C0000808B500F0B9F908BD5A
S31508005D5010B5FFF70DFE10B9FFF7B0FA10BDFEF744
S31508005D607DFA10B9FFF7AAFA10BDFFF75DFAFFF73B
S31508005D70C3FDFFF701FE20F0604020F07F00054BD1
S31508005D801860FFF7F9FD446800F09CF9A047FFF793
S31508005D9095FA10BD08ED00E070B508E0461C4D1CEC
S31508005DA00B780370FFF7E4F9224630462946531E5E
S31508005DB09CB2002AF2D170BDF0B5002421E0134D43
S31508005DC015F8147005EB440595F801E007EB0E0588
S31508005DD005FB00054AF2104C9CFBF5F605FB16C6BA
S31508005DE06EB99CFBF5F5ADB20D80013DADB2B5F5CA
S31508005DF0806F04D2177083F800E00120F0BD0134EB
S31508005E00E4B2112CDBD90020F0BD00BF349B00089A
S31508005E1010B582B001AB0DF105020DF106014FF484
S31508005E20FA70FFF7C9FF012804D040F2071151485C
S31508005E30FFF7B8FA504B00225A611A6842F400423A
S31508005E401A60FFF781FD00F1FA0405E0FFF790F903
S31508005E50FFF77AFD844204D3474B1B6813F4004FBF
S31508005E60F4D1454B1A6822F002021A601A6842F009
S31508005E7001021A60FFF768FD00F1FA0405E0FFF772
S31508005E8077F9FFF761FD844204D33B4B5B6813F057
S31508005E90010FF4D09DF805305A1E9DF80430013BD9
S31508005EA01B0543EA0243BDF80620013A1343324A6A
S31508005EB0D361136823F001031360FFF745FD00F172
S31508005EC0FA0405E0FFF754F9FFF73EFD844204D3D0
S31508005ED0294B5B6813F0010FF4D1284BD3F8002245
S31508005EE042F00102C3F80022D3F8002222F47C52C1
S31508005EF0C3F80022D3F8002242F46062C3F80022F5
S31508005F00D3F8002242F00102C3F80022D3F81C227B
S31508005F1022F48042C3F81C22D3F80C2242F48042B1
S31508005F20C3F80C22D3F8042222F48042C3F80422D0
S31508005F30134AC3F8B02202F14C520432C3F8B42211
S31508005F40D3F8042222F48042C3F80422D3F8142298
S31508005F5022F48042C3F81422D3F81C2242F4804269
S31508005F60C3F81C22D3F8002222F00102C3F800224B
S31508005F7002B010BD0C9B0008006800400064004099
S31508005F800000E0CC38B504460D46254B9B6813F057
S31508005F90806F04D140F28B112248FFF703FA204B99
S31508005FA0D3F8802102F00102C3F88021D3F88021BA
S31508005FB042F07C4242F40012C3F88021C3F88451AF
S31508005FC0E178A278120442EA0162617842EA012283
S31508005FD021780A43C3F88821E179A279120442EAB2
S31508005FE00162617942EA012221790A43C3F88C21C8
S31508005FF0D3F8802142F00102C3F88021FFF7A4FC00
S3150800600000F1320405E0FFF7B3F8FFF79DFC844280
S3150800601004D3034B9B6813F0806FF4D038BD00BFE0
S31508006020006800400C9B0008244BDB6813F0030F44
S3150800603041D0224BD3F8B03113F0040F04D11F4BD3
S31508006040D3F8B0315B0D05E01C4BD3F8B031DB0853
S3150800605043F0004340F26762934225D1174BD3F8C9
S31508006060B42102F00F020A70D3F8B8210270D3F8EF
S31508006070B821120A4270D3F8B821120C8270D3F8EC
S31508006080B821120EC270D3F8BC210271D3F8BC2114
S31508006090120A4271D3F8BC21120C8271D3F8BC31B2
S315080060A01B0EC371012000E00020044AD36843F0A8
S315080060B02003D36070470020704700BF0068004087
S315080060C072B6704762B670474278007840EA022096
S315080060D0704700BFC278837843EA0222437843EACE
S315080060E00223007840EA0320704700BF0170090ABE
S315080060F0417070470170C1F307234370C1F307432A
S315080061008370090EC170704713462AB10A78027067
S3150800611001300131013BF9D1704700BF01700130F0
S31508006120013AFBD1704700BF30B4451C03780878A4
S315080061301B1A013A04D04C1C28462146002BF4D0E1
S31508006140184630BC704700BF00E0013003780BB139
S315080061508B42FAD11846704702394369023B994285
S3150800616004D24389806A01FB030070470020704708
S3150800617070B506460D4601F11A00FFF7A5FF04465D
S315080061803378032B05D105F11400FFF79DFF44EA88
S31508006190004070BD70B506460C46154691B204F12E
S315080061A01A00FFF7A3FF3378032B04D1290C04F157
S315080061B01400FFF79BFF70BD2DE9F04180460F469E
S315080061C001F11A00FFF780FF50BB3D7805F03F0547
S315080061D06B1E03EB430503EB85050126002411E03E
S315080061E0174B185D3844FFF76FFF36B1FE2D1AD8E6
S315080061F028F815000646013503E04FF6FF73984266
S3150800620014D101340C2CEBD93B7813F0400F10D085
S31508006210FE2D11D8002328F815300120BDE8F0819D
S315080062200020BDE8F0810020BDE8F0810020BDE82F
S31508006230F0810120BDE8F0810020BDE8F08100BFB3
S31508006240EC9B00082DE9F84380460F4691464B73B0
S315080062500F23CB7200240C73214607F11A00FFF7AF
S3150800626045FF09F1FF3303EB430603EB8606254694
S315080062704FF6FF739D4202D038F8165001360C4B84
S31508006280185D29463844FFF731FF0DB94FF6FF75FB
S3150800629001340C2CECD94FF6FF739D4202D038F826
S315080062A016300BB949F0400987F80090BDE8F88325
S315080062B0EC9B000870B582B0054616461C460B22B4
S315080062C0FFF722FF052C12D814E0023600220CE054
S315080062D003F0010101EB44045B0814F4803F03D08A
S315080062E084F4883484F0210401320F2AF0D93388E3
S315080062F0002BEAD1072300E0134604F00F0202F14F
S315080063003001392901D902F137015A1E02A803447E
S3150800631003F8081C2409EFD17E210346134403F829
S31508006320081C002300E00133934202D2E95C2029CD
S31508006330F9D1591C2B44072A05D802A8104410F88D
S31508006340080C013200E0202018700B460729F0D906
S3150800635002B070BD0B210023DA0142EA530302782A
S3150800636052FA83F3DBB201300139F5D1184670478A
S31508006370016821B94FF0FF3316E0013200E00A4602
S3150800638013781F2B01D93A2BF7D13A2B0BD110B41E
S315080063904C1C0B78303B092B08D8A24209D15BB9B3
S315080063A0013202600AE00023184670474FF0FF33B7
S315080063B004E04FF0FF3301E04FF0FF3318465DF875
S315080063C0044B704738B50C4670B1054603685BB197
S315080063D01A784AB1D9888288914205D15878FDF74A
S315080063E029FC10F0010F03D000232360092038BDD3
S315080063F02B682360002038BDF8B5C37803B304467C
S31508006400C66A00F130070123324639464078FDF75F
S315080064104FFCB8B90023E370236AF31AA2699342C2
S3150800642012D2A57808E0A3691E44012332463946EC
S315080064306078FDF73DFC013D012DF4D80020F8BD3C
S315080064400020F8BD0120F8BD0020F8BD70B5C36A6C
S315080064508B4212D004460D46FFF7CEFF064668B9B2
S3150800646001232A4604F130016078FDF7F5FB10B1E7
S3150800647001264FF0FF35E56200E00026304670BD84
S3150800648010B504460023C3704FF0FF33C362FFF70D
S31508006490DDFFD8B904F22E20FFF716FE4AF655237B
S315080064A0984215D104F16600FFF714FE20F07F40EC
S315080064B00A4B98420ED004F18200FFF70BFE20F03B
S315080064C07F40064B984207D1002010BD042010BD1E
S315080064D0032010BD002010BD022010BD4641540007
S315080064E02DE9F04784B00E46174600230B60FFF7E8
S315080064F03FFF051EC0F22C81AA4B53F82540002CFD
S3150800650000F02881346007F0FE07237873B16078BD
S31508006510FDF790FB10F0010F08D1002F00F01C8149
S3150800652010F0040F40F01A81002038E10023237090
S31508006530E8B26070FDF766FB10F0010F40F01081BD
S315080065401FB110F0040F40F00D8100212046FFF71F
S3150800655097FF022815D0002628E004F130002B0109
S3150800656003F5DF73184403791BB10830FFF7B2FD52
S3150800657000E0002004AB03EB850343F8100C01355B
S3150800658000E00025032DE8D9002504AB03EB8503BD
S3150800659053F8106C26B131462046FFF771FF00E02C
S315080065A00320012802D90135032DEED9042800F06D
S315080065B0DB80012800F2DA8004F13B00FFF784FD56
S315080065C0B0F5007F40F0D48004F14600FFF77CFD6B
S315080065D0804620B904F15400FFF77CFD8046C4F8D4
S315080065E0188094F8409084F8029009F1FF33DBB2E2
S315080065F0012B00F2BF8008FB09F994F83D5065812C
S31508006600002D00F0B9806B1E1D4240F0B78004F1E2
S315080066104100FFF759FD8246208110F00F0F40F028
S31508006620AF8004F14300FFF74FFD074620B904F198
S315080066305000FFF74FFD074604F13E00FFF744FD03
S315080066400346002800F09E8009EB000202EB1A12AE
S315080066509742C0F09980BF1AB7FBF5F5002D00F0F8
S31508006660958040F6F5718D4201D8012700E0022792
S315080066704FF6F5718D4200D9032702356561E6614B
S31508006680334423623244A262032F0FD104F15A0025
S31508006690FFF71AFD00287BD1BAF1000F7AD104F171
S315080066A05C00FFF717FD6062AD000EE0BAF1000F5F
S315080066B072D04B446362022F01D16D0005E005EBF1
S315080066C0450305F0010505EB530505F2FF15B8EB83
S315080066D0552F63D34FF0FF332361E3608023237183
S315080066E0032F2CD104F16000FFF7EEFC012826D118
S315080066F0711C2046FFF7AAFE08BB0023237104F28B
S315080067002E20FFF7E1FC4AF65523984217D104F1EB
S315080067103000FFF7DFFC244B984210D104F50570D2
S31508006720FFF7D8FC214B984209D104F50670FFF70C
S31508006730D1FC206104F50770FFF7CCFCE0602770F8
S315080067401B4A138801339BB21380E380002026E09E
S315080067500B2024E00C2022E0002020E00A201EE086
S3150800676003201CE00A201AE0012018E00D2016E09C
S315080067700D2014E00D2012E00D2010E00D200EE093
S315080067800D200CE00D200AE00D2008E00D2006E0A3
S315080067900D2004E00D2002E00D2000E00D2004B0DD
S315080067A0BDE8F0878C1A002052526141727241612D
S315080067B0881A0020F8B50668012951D973699942E3
S315080067C050D20C463378022B2AD0032B37D0012B14
S315080067D04AD101EB5105316A01EB55213046FFF7E5
S315080067E035FE002842D16F1CC5F30805354495F8D7
S315080067F03050316A01EB57213046FFF727FE002853
S3150800680037D1C7F308073E4496F8300045EA00201A
S3150800681014F0010F01D00009F8BDC0F30B00F8BD54
S31508006820316A01EB14213046FFF710FE20BB6000E9
S3150800683000F4FF7030303044FFF746FCF8BD316A8B
S3150800684001EBD4113046FFF701FEC0B9A00000F4F1
S31508006850FE7030303044FFF73DFC20F07040F8BD44
S315080068600120F8BD0120F8BD0120F8BD4FF0FF302A
S31508006870F8BD4FF0FF30F8BD4FF0FF30F8BD4FF0D0
S31508006880FF30F8BD2DE9F0410768B1F5001F3DD28C
S3150800689006460C4611F01F0F3BD1316185681DB9BC
S315080068A03B78022B00D97D6A35B93B89B3EB541F77
S315080068B032D97B6AB3611AE0B7F80A804FEA4828EA
S315080068C00EE029463046FFF775FF0546B0F1FF3F53
S315080068D025D0012826D97B69984226D2C8EB04041C
S315080068E04445EED229463846FFF736FCB061756155
S315080068F0B369EBB103EB5423B36107F13003C4F377
S3150800690008042344F3610020BDE8F0810220BDE8B5
S31508006910F0810220BDE8F0810220BDE8F081012067
S31508006920BDE8F0810220BDE8F0810220BDE8F081D3
S315080069300220BDE8F08100BF2DE9F843012979D985
S315080069404369994278D217460C4605460378022BC6
S3150800695044D0032B54D0012B70D101EB5108016AA6
S3150800696001EB5821FFF772FD0646002867D108F1AA
S315080069700109C8F3080814F001040BD005EB080355
S3150800698093F830203B0103F47F6302F00F021343B0
S31508006990DBB200E0FBB2A84488F830300123EB7084
S315080069A0296A01EB59212846FFF750FD06460028BB
S315080069B045D1C9F3080914B1C7F3071208E005EB76
S315080069C0090393F8303023F00F03C7F303221A4361
S315080069D0A94489F830200123EB7030E0016A01EB05
S315080069E01421FFF733FD064648BB600000F4FF702C
S315080069F03030B9B22844FFF779FB0123EB701EE06B
S31508006A00016A01EBD411FFF721FD0646B8B927F054
S31508006A107047A40004F4FE7430342C442046FFF773
S31508006A2059FB00F0704139432046FFF763FB012309
S31508006A30EB7004E0022602E0022600E00226304659
S31508006A40BDE8F8832DE9F04107460668884629B966
S31508006A50F5687DB173699D420ED20EE0FFF7AAFE76
S31508006A60012846D9B0F1FF3F51D0736998424ED3F9
S31508006A70454602E0012500E001252C4601347369EC
S31508006A809C4202D3012D37D9022421463846FFF706
S31508006A9091FE38B1012832D0B0F1FF3F31D0AC4277
S31508006AA0ECD130E04FF0FF3221463046FFF744FF85
S31508006AB0034640B9B8F1000F05D022464146304694
S31508006AC0FFF73AFF034673B9F46033697269023A0D
S31508006AD0934201D2013B3361337943F001033371A9
S31508006AE02046BDE8F081012B10D14FF0FF30BDE8FC
S31508006AF0F0810120BDE8F0810020BDE8F081BDE805
S31508006B00F081BDE8F0810020BDE8F0810120BDE8F4
S31508006B10F08100BFF8B50E46046801292CD907464E
S31508006B20114663699E4229D22AB14FF0FF322046A8
S31508006B30FFF702FF20BB31463846FFF73BFE054606
S31508006B40F8B101281FD0B0F1FF3F1ED00022314610
S31508006B502046FFF7F1FED0B92369B3F1FF3F05D010
S31508006B6001332361237943F00103237163692E46B8
S31508006B709D42E0D30020F8BD0220F8BD0220F8BDF2
S31508006B80F8BD0020F8BD0220F8BD0120F8BDF8BD0B
S31508006B902DE9F8430668036903F120058369002B8C
S31508006BA06ED0B5F5001F6ED288460446C5F30807B1
S31508006BB0002F5DD101338361416941B93389B3EB54
S31508006BC0551F55D8002383610420BDE8F8837389CF
S31508006BD0013B13EA55234BD1FFF7ECFD814601280B
S31508006BE054D9B0F1FF3F54D07369984239D3B8F1FC
S31508006BF0000F04D10023A3610420BDE8F88361696E
S31508006C002046FFF71FFF8146002845D0012846D0B9
S31508006C10B0F1FF3F46D03046FFF7EEFB002844D1DF
S31508006C204FF40072002106F13000FFF777FA494663
S31508006C303046FFF791FAF0624FF000080AE00123A8
S31508006C40F3703046FFF7D8FB90BB08F10108F36AEA
S31508006C500133F36273899845F1D3F36AC8EB0303EA
S31508006C60F362C4F8149049463046FFF775FAA061F6
S31508006C70256107F130084644E6610020BDE8F8833F
S31508006C800420BDE8F8830420BDE8F8830220BDE8A7
S31508006C90F8830120BDE8F8830720BDE8F8830220C1
S31508006CA0BDE8F8830120BDE8F8830120BDE8F88334
S31508006CB00120BDE8F88300BFF8B504460F4606680C
S31508006CC00021FFF7DFFD0246B8B90025A169304665
S31508006CD0FFF7BCFB024680B9E3691B78E52B00D0B9
S31508006CE01BB90135BD4201D107E000250121204627
S31508006CF0FFF74EFF02460028E8D0042A00D10722F3
S31508006D001046F8BD2DE9F8430446884607684FF053
S31508006D10FF094E4604254CE03846FFF797FB054623
S31508006D2000284BD1E1690A78002A46D0CB7A03F0CD
S31508006D303F03A371E52A2BD02E2A2BD023F020005F
S31508006D40082814BF00200120404525D10F2B15D156
S31508006D5012F0400F06D091F80D9002F0BF02236999
S31508006D6063621646B24219D14B7B994518D1A06A7F
S31508006D70FFF722FAB0B1013EF6B214E026B908468A
S31508006D80FFF7E8FA814519D04FF0FF33636215E043
S31508006D90FF2608E0FF2606E0FF2604E0FF2602E0BD
S31508006DA0FF2600E0FF2600212046FFF7F1FE0546F4
S31508006DB020B9A1690029AFD100E004250DB100234F
S31508006DC0A3612846BDE8F88370B5044605680669D8
S31508006DD0416AB1F1FF3F03D0FFF754FD034600E0D7
S31508006DE00023BBB9A1692846FFF730FB034670B9F3
S31508006DF0E269E52111700122EA702269964206D9F4
S31508006E0000212046FFF7C4FE03460028EAD0042BDB
S31508006E1000D10223184670BD2DE9F04F83B006460F
S31508006E208A46D1F80090856A002423465F1C19F823
S31508006E3003001F2805D92F2803D05C280AD100E0B3
S31508006E40013709EB070219F807302F2BF8D05C2B0E
S31508006E50F6D017E0FE2C00F2E280012100F0D6FF02
S31508006E608046002800F0DD807F2806D80146714854
S31508006E70FFF76AF9002840F0D68025F814803B46CB
S31508006E800134D3E7CAF800201F2802D84FF00408B7
S31508006E900CE04FF0000809E004F10043013B35F827
S31508006EA01330202B01D02E2B02D1013C002CF3D11C
S31508006EB0002325F81430002C00F0B7800B2220217F
S31508006EC0306AFFF72BF9002300E0013335F8132069
S31508006ED0202AFAD02E2AF8D01BB148F0030800E081
S31508006EE0013C6CB104F10042013A35F812202E2A11
S31508006EF0F6D14FF0080B4FF0000ACDF804A005E0D4
S31508006F004FF0080B4FF0000ACDF804A003F1010971
S31508006F1035F81370002F57D0202F03D02E2F05D108
S31508006F204C4503D048F003084B46EFE7DA4501D253
S31508006F304C4515D1BBF10B0F02D148F0030843E0CD
S31508006F404C4501D048F003084C453DD3019B9B00B6
S31508006F50DBB2019323464FF00B0B4FF0080AD5E737
S31508006F607F2F0BD90021384600F050FF074618B18D
S31508006F70A0F18007304BDF5D48F0020827B139469B
S31508006F802E48FFF7E1F818B148F003085F2714E028
S31508006F90A7F141039BB2192B04D8019B43F00203C6
S31508006FA001930AE0A7F161039BB2192B05D8019B4F
S31508006FB043F001030193203FBFB2336A03F80A7016
S31508006FC04B460AF1010AA1E7336A1A78E52A01D184
S31508006FD005221A70BBF1080F03D1019B9B00DBB297
S31508006FE00193019901F00C020C2A03D001F0030366
S31508006FF0032B01D148F0020818F0020F0AD1019BB1
S3150800700003F00303012B01D148F01008042A01D12B
S3150800701048F00808336A83F80B80002006E006204B
S3150800702004E0062002E0062000E0062003B0BDE8E2
S31508007030F08F00BF589B00086C9B0008649B0008F3
S31508007040F8B500238B758369002B69D00D46064673
S31508007050436AB3F1FF3F17D0836A002409E0002191
S3150800706000F0D4FE50B1FE2C0AD82A1990753B467A
S3150800707001349F1C18880028F1D102E0002400E0A2
S3150800708000242C440023A375AC7D0022134628E077
S31508007090F069591CC35C202B22D0052B00D1E523AF
S315080070A0092907D114B9A8182E278775A8182E27D5
S315080070B047720132A81843728CB9A3F14100C0B2D5
S315080070C019280AD8F069007B082901D9102700E099
S315080070D00827074201D02033DBB2A818837501328E
S315080070E00B460A2BD4D934B9AB1800219975F36924
S315080070F01B7B03B90A462A4400235372F369DB7AD9
S315080071002B72F0691C30FEF7E5FF2860F06918302D
S31508007110FEF7DAFFA880F0691630FEF7D5FFE8809B
S31508007120F8BD00BF2DE9F0478146884601F11A00EF
S31508007130FEF7CAFFA8BB98F8005005F03F056B1E7E
S3150800714003EB430503EB8505012700241BE01F4BD2
S31508007150185D4044FEF7B8FF06467FB1FE2D23D8DA
S3150800716000F072FE074605F1010A39F8150000F02D
S315080071706BFE87421BD13746554603E04FF6FF7331
S31508007180984217D101340C2CE1D998F8003013F045
S31508007190400F12D0A7B139F81530A3B90120BDE8C0
S315080071A0F0870020BDE8F0870020BDE8F0870020C2
S315080071B0BDE8F0870020BDE8F0870120BDE8F0872C
S315080071C00120BDE8F0870020BDE8F087EC9B0008A9
S315080071D02DE9F8430446D0F800800021FFF752FB5A
S315080071E000285CD14FF0FF3363624FF0FF094F462A
S315080071F0A1694046FFF72AF90646002851D1E569F4
S315080072002B78002B4FD0E97A01F03F02A271E52BCB
S3150800721004D011F0080F06D00F2A04D04FF0FF3320
S315080072206362FF2733E00F2A17D1A06A78B313F0F9
S31508007230400F06D095F80D9003F0BF0322696262ED
S315080072401F46BB421ED16B7B99451DD12946FFF7C8
S3150800725069FFD8B1013FFFB219E027B92846FFF701
S3150800726079F8814522D0216ACB7A13F0010F04D12F
S315080072700B222846FEF758FFD8B14FF0FF3363625A
S31508007280FF2704E0FF2702E0FF2700E0FF27002191
S315080072902046FFF77DFC0028AAD0BDE8F883BDE8A4
S315080072A0F883BDE8F8830420BDE8F8833046BDE8D6
S315080072B0F8833046BDE8F88330B583B004460191BB
S315080072C0056801E001330193019B1A782F2AF9D04A
S315080072D05C2AF7D00022A2601B781F2B08D8236AE5
S315080072E08022DA7200212046FFF7CCFA034626E010
S315080072F001A92046FFF790FD034600BB2046FFF78D
S3150800730067FF236ADA7A034628B1042817D112F0F0
S31508007310040F11D013E012F0040F10D1A37913F063
S31508007320100F0BD02169C1F30801303129442846D2
S31508007330FEF71EFFA060DBE7052300E005231846DD
S3150800734003B030BD2DE9F04784B00668D0F820A018
S31508007350D0F828809AF80B3013F0A00F40F08380FD
S31508007360002400E0013438F81430002BFAD1054621
S315080073700C22514601A8FEF7C7FE9DF80F3013F000
S31508007380010F1ED000238AF80B30AB6201270BE0F1
S315080073903B46424601A95046FEF78CFF2846FFF7B2
S315080073A017FF814610B90137632FF1D9642F5CD0D6
S315080073B0B9F1040F5BD19DF80F308AF80B30C5F888
S315080073C028809DF80F3013F0020F06D00C342B4B93
S315080073D0A3FB0434A408013400E00124214628460E
S315080073E0FFF76AFC034618BB013C21D02969A1EBCB
S315080073F044112846FFF746FA0346C8B9286AFEF735
S31508007400A9FF0746A9693046FFF720F8034678B969
S315080074103B46E2B2E969A86AFEF714FF0123F37056
S3150800742000212846FFF7B4FB034608B9013CE9D119
S31508007430FBB9A9693046FFF709F88146D8B9202271
S315080074400021E869FEF76AFE0B22296AE869FEF759
S315080074505BFEEA692B6ADB7A03F0180313730123D0
S31508007460F370484607E0062005E0072003E0484693
S3150800747001E01846FFE704B0BDE8F0874FECC44EBC
S3150800748070B50446FEF7B8FF0546002837D12378BD
S31508007490032B2DD12379012B2AD104F130064FF481
S315080074A0007200213046FEF739FE4AF6552104F2ED
S315080074B02E20FEF71BFE13493046FEF71BFE124927
S315080074C004F50570FEF716FE216904F50670FEF749
S315080074D011FEE16804F50770FEF70CFEE269013259
S315080074E0E262012331466078FCF7E2FB0023237150
S315080074F0002211466078FCF707FC00B101252846F2
S3150800750070BD00BF525261417272416110B584B0BC
S3150800751001900091144604A840F8041DFEF728FFC0
S31508007520002816DB0E4B53F820300BB100221A70D8
S31508007530019B0BB100221A70019B094A42F82030C0
S315080075404BB1012C09D1002201A96846FEF7C8FFF4
S3150800755004E00B2002E0002000E0002004B010BD8B
S315080075608C1A00202DE9F04393B00191002800F011
S31508007570AA80054616460023036002F01F073A460E
S3150800758006A901A8FEF7ACFF002840F09E80069BDE
S31508007590079303AB0F934F4B1193019907A8FFF776
S315080075A08BFE044628B90F9B93F90B30002B00DAA3
S315080075B0062416F01C0F53D044B1042C03D107A897
S315080075C0FFF7C0FE044647F008070BE09DF8223097
S315080075D013F0110F03D116F0040F02D102E00724AD
S315080075E000E00824002C4BD117F0080F48D03A4E7B
S315080075F031460E980E30FEF77DFD31460E98163050
S31508007600FEF778FD20220E9BDA72069EDDF838809A
S3150800761041463046FEF7ACFD8146002241463046DB
S31508007620FEF7B8FD00210E981C30FEF763FD012217
S31508007630069BDA70B9F1000F22D0069BDE6A00229B
S31508007640494607A8FFF766FA0446C8B931460698B8
S31508007650FEF7FCFE044609F1FF33069AD3600FE0F5
S3150800766074B99DF8223013F0100F06D116F0020FE8
S3150800767006D013F0010F02D102E0042400E007242B
S315080076804CB917F0080F01D047F02007069BDB6AB4
S315080076902B620E9B6B62CCB9069EDDF8388041469C
S315080076A03046FEF765FDA86008F11C00FEF712FDDE
S315080076B0E86000236B746B61EB612F742E60F388AE
S315080076C0AB80204603E0092001E000E0204613B025
S315080076D0BDE8F08388180020000061482DE9F04FC6
S315080076E083B00446884615461F4600233B6001A919
S315080076F0FEF768FE002840F0A280607C002840F073
S31508007700A080237C13F0010F00F09A80E668636975
S31508007710F61AAE42C0F08E802E468BE06369C3F33C
S315080077200802002A70D1019A5289013A12EA5329AD
S3150800773012D10BB9A06803E0A1692046FFF73AF811
S31508007740012802D8022060747BE0B0F1FF3F02D125
S315080077500120607475E0A061DDF804A0A1695046B7
S31508007760FEF7FAFC054610B90220607469E04D443C
S315080077705FEA562B25D009EB0B03BAF80A20934289
S3150800778001D9C9EB020B5B462A4641469AF8010025
S31508007790FCF762FA10B10120607452E0237C13F002
S315080077A0400F0BD0E069401B834507D94FF40072A0
S315080077B004F1280108EB4020FEF7A6FC4FEA4B250A
S315080077C030E0E26995421ED0237C13F0400F0ED0BC
S315080077D0012304F128019AF80100FCF769FA10B1AF
S315080077E0012060742DE0237C23F0400323740123D9
S315080077F02A4604F1280101984078FCF72DFA10B1C1
S31508007800012060741DE0E5616169C1F30801C1F5F5
S315080078100075AE4200D2354628312A4621444046F4
S31508007820FEF772FCA84463692B4463613B682B44EA
S315080078303B60761B002E7FF471AF002001E000E06C
S31508007840072003B0BDE8F08F2DE9F04F83B004465A
S31508007850884616461F4600233B6001A9FEF7B2FD7F
S31508007860002840F0BE80607C002840F0BC80237C65
S3150800787013F0020F00F0B6806369F342C0F0A880E7
S31508007880DE43A5E06369C3F30802002A40F081805D
S31508007890019A5289013A12EA53291DD133B9A068CF
S315080078A040B900212046FFF7CDF803E0A16920463C
S315080078B0FFF7C8F8002800F08E80012802D10220C0
S315080078C0607490E0B0F1FF3F02D1012060748AE055
S315080078D0A061A36803B9A060237C13F0400F0FD002
S315080078E00123E26904F1280101984078FCF7E0F9E0
S315080078F010B10120607476E0237C23F040032374E2
S31508007900DDF804A0A1695046FEF726FC054610B925
S315080079100220607467E04D445FEA562B25D009EBD8
S315080079200B03BAF80A20934201D9C9EB020B5B464E
S315080079302A4641469AF80100FCF7BAF910B1012027
S31508007940607450E0E169491B8B450BD94FF400720E
S3150800795008EB412104F12800FEF7D6FB237C23F02F
S31508007960400323744FEA4B2525E0E3699D420FD077
S315080079706269E3689A420BD201232A4604F1280178
S315080079809AF80100FCF768F910B1012060742AE042
S31508007990E5616069C0F30800C0F50075AE4200D223
S315080079A0354628302A4641462044FEF7ADFB237C5F
S315080079B043F040032374A84463692B446361E26877
S315080079C0934238BF1346E3603B682B443B60761B03
S315080079D0002E7FF457AF237C43F020032374002046
S315080079E001E000E0072003B0BDE8F08F70B582B073
S315080079F004460E460A2902D10D21FFF7F7FF6368F0
S31508007A00002B16DB5D1C23441E733C2D0DDD01ABDC
S31508007A102A4604F10C012068FFF716FF019B9D42D8
S31508007A2001D1002501E04FF0FF356560A3680133F9
S31508007A30A36002B070BD00BF30B583B0044601A98B
S31508007A40FEF7C0FC00283CD1227C12F0200F39D06A
S31508007A5012F0400F0CD00123E26904F128010198C5
S31508007A604078FCF725F970BB237C23F04003237488
S31508007A70216A0198FEF7EAFC38BB656AEB7A43F09F
S31508007A802003EB72A26829462068FEF783FBE168AB
S31508007A9005F11C00FEF72EFB0D4905F11600FEF751
S31508007AA029FB002105F11200FEF720FB0122019BAC
S31508007AB0DA700198FFF7E4FC237C23F02003237493
S31508007AC003E002E001E00120FFE703B030BD00BF9C
S31508007AD00000614810B582B00446FFF7ADFF0346C3
S31508007AE038B901A92046FEF76DFC034608B90022FD
S31508007AF02260184602B010BDF0B583B004460E46A3
S31508007B0001A9FEF75FFC002840F0A480657C002DE3
S31508007B1040F0A180E368B34204D2227C12F0020F3F
S31508007B2000D11E46636900226261002E5DD0019A6B
S31508007B3057897F026BB1721EB2FBF7F2013BB3FBAA
S31508007B40F7F18A4205D37A4213406361F61AA169AE
S31508007B5012E0A16879B92046FEF774FF01460128AC
S31508007B6002D10220607479E0B0F1FF3F02D1012012
S31508007B70607473E0A060A16119BB002638E0237C1D
S31508007B8013F0020F05D02046FEF75CFF014620B928
S31508007B901AE02046FEF70EFE0146B1F1FF3F02D17C
S31508007BA0012060745AE0012903D9019B5B69994257
S31508007BB002D30220607451E0A16163693B446361AA
S31508007BC0F61BBE42DBD800E03E4663693344636178
S31508007BD0C6F308035BB10198FEF7BEFA10B9022096
S31508007BE060743BE000EB562602E0002600E0002623
S31508007BF06369C3F3080313B3E26996421FD0237C73
S31508007C0013F0400F0ED0012304F1280101984078A3
S31508007C10FCF74EF810B1012060741FE0237C23F0B6
S31508007C20400323740123324604F128010198407861
S31508007C30FCF712F810B1012060740FE0E661636981
S31508007C40E268934209D9E360237C43F02003237456
S31508007C50284603E002E0284600E0284603B0F0BDC7
S31508007C6030B591B001900D46002205A901A8FEF78E
S31508007C7037FC0446A8B902AB0D930B4B0F93019939
S31508007C8005A8FFF719FB044658B90D9B93F90B3065
S31508007C90002B05DB2DB1294605A8FFF7D1F900E031
S31508007CA00624204611B030BD8818002070B59CB057
S31508007CB00190022205A901A8FEF712FC059B119363
S31508007CC0044600284AD102AB1993264B1B93019907
S31508007CD011A8FFF7F1FA044600283FD1199B93F93A
S31508007CE00B30002B05DB9DF84A3013F0010F02D14B
S31508007CF002E0062400E00724ECB9059E18993046F0
S31508007D00FEF736FA05469DF84A3013F0100F13D0E1
S31508007D1006960890002106A8FEF7B4FD044658B951
S31508007D20002106A8FEF7EEFF034600B90723042B39
S31508007D3002D01C4600E0002584B911A8FFF744F8D4
S31508007D40044630B92DB10022294611A8FEF7E2FEF5
S31508007D5004461CB90598FFF793FB044620461CB059
S31508007D6070BD00BF881800202DE9F04182B080461A
S31508007D700E4617460546002412E06B46012201A965
S31508007D803846FFF7ABFC009B012B0ED19DF804305B
S31508007D900D2B05D06A1C2B7001340A2B04D015460E
S31508007DA0731E9C42E9DB00E0154600232B700CB9D4
S31508007DB0184600E0404602B0BDE8F08110B594B020
S31508007DC00446019100230293039303E0013401A8BA
S31508007DD0FFF70CFE21780029F8D1029A002A0BDB5E
S31508007DE06B4604A90198FFF72FFD40B9009B029A3C
S31508007DF09A4207D1039807E04FF0FF3004E04FF0AE
S31508007E00FF3001E04FF0FF3014B010BD7F2817D9BE
S31508007E1079B1FF2813D8A0F180030A4A32F8130073
S31508007E207047084A32F81320904205D001339BB2B6
S31508007E3000E000237F2BF4D98033D8B270470020A6
S31508007E40704700BFAC9E0008F0B4B0F5805F01D261
S31508007E50204B02E0204B00E02B461A88002A36D039
S31508007E60904234D31D1D5B88190ADBB29C18A042C8
S31508007E7028DA08292BD8DFE801F005090F121518AA
S31508007E801B1E2100861A35F8160020E0821A02F019
S31508007E900103C01A80B21AE0103880B217E0203801
S31508007EA080B214E0303880B211E01A3880B20EE0A1
S31508007EB0083080B20BE0503880B208E0A0F5E350F5
S31508007EC080B204E00029C7D105EB4303C5E7F0BC3F
S31508007ED0704700BFB89C0008FC9B000810B4013A24
S31508007EE00A440BE00C784B7803EB04239BB2184446
S31508007EF080B2834201D9013080B202319142F1D376
S31508007F0007D10B781B02184480B2834201D901308D
S31508007F1080B25DF8044B704770B4C5780D44EDB275
S31508007F20134CE57083780E0A3344DBB2A3704278AB
S31508007F306270007820709CB2A64206D90132D2B28D
S31508007F400B4C62700AB901302070C9B28D420CDA46
S31508007F500133DBB2064A93703BB953780133DBB27F
S31508007F60537013B913780133137070BC704700BF90
S31508007F70182A002010B5094C2368014603F10800A9
S31508007F80FFF7CAFF2368064A1178197251785972A1
S31508007F9091789972D278DA7210BD00BF282A00202B
S31508007FA0182A002000221A4B1A7006E00021194AE6
S31508007FB022F813100133164A1370154B1B78002B41
S31508007FC0F4D00022124B1A7008E06822124902FB0C
S31508007FD003120021517601330D4A13700C4B1B789E
S31508007FE0002BF2D04FF480620C4B1A800022084B0B
S31508007FF01A7007E00A4A02EB8312002191800133C6
S31508008000034A1370024B1B78002BF3D0704700BF4E
S315080080109A1A0020942A00202C2A0020981A002058
S31508008020E830002000220A4B1A700BE01946094A6C
S3150800803032F813201AB9074B23F811007047013399
S31508008040034A1370024B1B78002BEFD0704700BF12
S315080080509A1A0020942A0020030A43EA002080B2D4
S31508008060704700BF08B5142205490020FFF736FF00
S3150800807010B1FFF7F1FF08BD4FF6FF7008BD00BF4E
S31508008080B22A002038B50D4D2C7C6B7C03EB0424FA
S31508008090143CA4B22044082205F11A0180B2FFF765
S315080080A01DFF224605F12201FFF718FF10B1FFF761
S315080080B0D3FF38BD4FF6FF7038BD00BFA42A002095
S315080080C008B50620FFF7DEFF08BD00BF70B5A54B53
S315080080D01C68042800F07181A34BA44A1360A44AC3
S315080080E01360032810D1637E03F00F03032B40F0BF
S315080080F0D285238A002B40F0CE8508229D4B1A7024
S31508008100FCF75AFC00F08CBC02287BD19A4AD3783B
S315080081100133DBB2D37063B993780133DBB2937062
S315080081203BB953780133DBB2537013B91378013373
S3150800813013700023914A1380914A1380637E072B9C
S3150800814001D0052B0AD1A37E0133DBB2A376782BA7
S3150800815040F0A1850023637600F09DBD002B00F05A
S315080081609A85228A002A41D0A27E511EA176002A2B
S3150800817040F09185E27E082A05D0591EC9B2012928
S315080081800ED8052A0CD1002363768022794B1A7003
S31508008190FCF712FC14227B4B83F82F2000F00CBD51
S315080081A0042A03D803219140C9B200E03021A17600
S315080081B00132E27603F00F03013B072B00F26B85D1
S315080081C0DFE813F0740208000D00EA036905EA0304
S315080081D06905EA0300226B4B83F82F206AE2042222
S315080081E0644B1A70FCF7E8FB00F04FBC03F00F0372
S315080081F0032B40F0508508225E4B1A70FCF7DCFB17
S3150800820000F00EBC052817D15F4B1B689B88002B16
S3150800821000F041850023534A13605C4A53490A60BB
S3150800822053490A60564A1380544A13800822514B10
S315080082301A7001F021FAC0E0524B9B7B452B40F0A7
S315080082402A85504A157C537C03EB05214B4A128834
S31508008250914200F320858DB2484B1D80494B1B7D0A
S3150800826013F03F0F40F01785464B5B7D002B40F01F
S315080082701285474B1C880CB95B885BB1414BDB8B7D
S315080082809C4240F008853F4B1A8C414B5B889A42CA
S3150800829040F00185FFF7E6FE4FF6FF73984240F07F
S315080082A0FA84384BDB7D062B00F0B880112B23D0DF
S315080082B0012B40F0F084334B93F82230082B40F022
S315080082C0EA84304B002283F822209B8C4FF6F67204
S315080082D0934203D909332B4A938402E00833294A87
S315080082E09384284B5A8BDA839A8B1A845C83284AA0
S315080082F052889A8300F0CBBC1C3D204B1D80254A32
S31508008300214B1A6026E09A880AB31E49898C8A424C
S315080083101DD1DA8832B11B49498C8A4202D0B2F59E
S315080083208A4F14D11A8812B95988002936D04FF6BF
S31508008330FF718A4202D1588888422FD01149498B49
S315080083408A4204D10F4A918B5A88914226D04033EB
S315080083500D4A13600C4B1B680F4A9342D3D300F0A7
S315080083609ABC00BF282A0020DA2A0020242A0020E6
S31508008370142A00201C2A0020941A0020102A002003
S31508008380E6300020A42A0020202A0020CE2A002039
S31508008390A02A0020E8300020283100200023AC4A1B
S315080083A013600221AB4A1170AB4AAC490A60AC496A
S315080083B00A60AC4A138001F05FF9AA4B1A88002AB2
S315080083C000F0698402F11C0189B2A74B1980A74BFA
S315080083D0080A18745974A6490968087A9875112004
S315080083E0D875083292B2100A40EA0222DA840022CC
S315080083F083F8282083F829208A885A84CA889A8488
S315080084009C4A1088588352889A830A88DA834A884D
S315080084101A843633914A136000F024BCFFF750FEE5
S315080084204FF6FF73984240F03684934C17E0617E0E
S31508008430A1B18E4B9A8CA3889A420FD18B4B5A8C3A
S31508008440E3889A420AD1894B5A8B23889A4205D1E6
S31508008450864B9A8B63889A4200F046816834864B2D
S315080084609C42E4D9814B93F82F3003F03F03022B4B
S3150800847014D17E4B9B8C99B2804A13800022804B84
S315080084801A7007E07F4A32F8132091425BD0013315
S315080084907B4A13707A4B1B78002BF3D0734B93F8F7
S315080084A02F3013F0040F40F0F683704B142283F834
S315080084B02F2028216C4A1180502283F82E2093F809
S315080084C0290093F82D2083F8292093F8281093F88B
S315080084D02C2083F8282083F82C1093F8272093F86B
S315080084E02B4083F8274083F82B2093F82640644DC9
S315080084F02C7093F82A5083F8265083F82A400130C6
S31508008500C0B283F82D0068B94B1CDBB2574981F815
S315080085102C303BB9531CDBB281F82B3013B901342C
S3150800852081F82A40514B5A8C54490A80998C5984AF
S315080085309A845A8BDA839A8B1A844E4A11885983FD
S3150800854052889A8379E300244D4B1C701CE0194627
S315080085506822494802FB0302527E1AB9682404FBC2
S31508008560010415E0072A0CD13CB16822424902FBF6
S315080085700312917EA27E914203D93F4A682404FBE6
S31508008580032401333E4A13703D4B1B78002BDED083
S31508008590002C00F080832E4B1C600323A3762376E1
S315080085A00023A3750422E275E376304DAB8CA380D5
S315080085B06B8CE3806B8B2380AB8B638001206076AA
S315080085C0314B1A7822735A7862739A78A273DB78D9
S315080085D0E373208295F82930E37295F82830A37260
S315080085E095F82730637295F826302372FFF7C2FC98
S315080085F095F82E0000F0F003502B57DD0022204B93
S315080086001A704BE003F13602184DAA5C002A4DD0C9
S31508008610012A03D101331A4A13703FE0022A35D1E1
S3150800862003F13702114DAA5C042A2FD101F1380350
S31508008630EA5C39316B5C43EA0222104B1A8040F23D
S315080086400A63934228BF13466382A3822EE000BFC3
S31508008650282A00201C2A0020CE2A0020242A0020AE
S31508008660142A0020E6300020102A0020A42A002020
S31508008670202A0020A02A00202C2A0020901A002058
S315080086809A1A0020942A0020941A002003F137022F
S31508008690A6498A5C52B11344A54A1370A44B1B78A9
S315080086A019460209053AB3EB820FABDB10229F4B42
S315080086B083F82F209D4B93F82F2042F0020283F86F
S315080086C02F20022283F83620042283F83720062238
S315080086D083F838200A2283F839202C21954A1180FC
S315080086E0602283F82E206EE2934B1C600022934B87
S315080086F01A708E4B93F82F2012F0040F07D0002320
S31508008700637620228D4B1A70FCF756F9C3E2874B25
S3150800871093F82E301B099B0085480370EB1A143B0F
S315080087209BB28448038001F00F01022903D102F0AD
S315080087303F0112290FD013B912F0030F0BD07B4B50
S31508008740D98C2389994240F03382784B198D6389F5
S31508008750994240F02D8212F0100F47D0218A002945
S3150800876044D004F10C00FFF7D7FB704B93F82A307E
S31508008770734A1078834239D16C4B93F82B30517871
S315080087808B4233D1694B93F82C30927893422DD192
S31508008790664B93F82D506A4BDB789D4226D12073A1
S315080087A06173A273E373E37ECBB9237EA27E9B1A21
S315080087B0DBB2A17DA3EBD103DBB25AB21944C9B22D
S315080087C0A175002A01DA5B425AB2E37DA2EB930255
S315080087D053FA82F2D3B2E37503EBD103237601226F
S315080087E0564B1A70237EA37600232382617E01F0FE
S315080087F00F03013B072B00F24E82DFE813F0080057
S315080088002300A7007301A301BF01D90165014B4BE2
S315080088101B7813F0010F00F03E8203236376402293
S31508008820464B1A7000232382424B188820B14222F5
S31508008830424B1A70FFF79EFB0022424B1A80FCF748
S31508008840BBF8EDE03D4B1B7813F0010F63D0374BB7
S3150800885093F82F3003F03F03122B5CD1334B93F878
S315080088602E0000F0F003502B37DD0022304B1A7033
S315080088702BE003F136022D4DAA5C72B3012A03D10F
S3150800888001332B4A137020E0022A16D103F137026E
S31508008890264DAA5C042A10D101F13803EA5C393165
S315080088A06B5C43EA0222284B1A8040F20A63934221
S315080088B028BF13466382A3820FE003F137021B49E0
S315080088C08A5C52B113441A4A1370194B1B7819461D
S315080088D00209053AB3EB820FCBDB03236376134B0E
S315080088E093F82620227293F82720627293F828209C
S315080088F0A27293F82930E3720120FFF73BFB42226C
S315080089000E4B1A70002323820A4A13800D4A1380DD
S31508008910FCF752F884E02022084B1A70FCF74CF852
S31508008920054B1B6800225A76B8E500BFA42A00202A
S315080089309A1A0020102A0020282A00201C2A002023
S31508008940182A0020E6300020901A0020914B93F850
S315080089502F3013F0010F24D011F0100F21D1238AE4
S31508008960002B40F098818C4D2888013080B2FFF7A3
S3150800897001FB8A4A137843F0100313702A881AB148
S3150800898043F00203854A1370FCF716F80123238285
S31508008990082363760023E37611227E4B83F82F2083
S315080089A00AE113F0200F10D07A4890F834301A02F2
S315080089B090F8353043EA0200794D2E683044286035
S315080089C0754813430288D31A0380734B188848B135
S315080089D011F0100F06D1714A137843F00203137091
S315080089E0FFF7C8FA6B4A92F8301092F8313003EB69
S315080089F001239BB26B4A1380A28A934200D80BB913
S31508008A00684B1A80674B1B886382644B1B7813F08C
S31508008A10030F00F040810022634B1A80FBF7CCFF5E
S31508008A205E4B1B7813F0200F08D000235E4A138094
S31508008A3063761422574B83F82F20BDE013F0100FEE
S31508008A400CD00023584A138001222282042262761F
S31508008A50E37611224F4B83F82F20ADE0524A128855
S31508008A608AB113F0010F01D000232382238A43B968
S31508008A70638A9A4201D94C4A13804B4B1B8823823E
S31508008A8001E0494A13800023E376484B1A68444BB1
S31508008A901A60454B1B884BB1238A3BB128333E4AA3
S31508008AA0138018223B4B83F82F2088E03B4B1B781A
S31508008AB013F0020F00F0EF802822374B1A8010229D
S31508008AC0344B83F82F207AE0344B1B7813F0010FD0
S31508008AD000F0E180002363761022304B1A70FBF712
S31508008AE06BFFD8E02C4B188808B1FFF743FA294BDF
S31508008AF093F82F3013F0010F15D0284B1B7813F07D
S31508008B00010F05D0072363760023A376238201E0AD
S31508008B10062363760120FFF72DFA10221F4B1A70E1
S31508008B20FBF74AFF44E01D4B1B7813F0010F04D0F6
S31508008B300523637600232382ADE0174B1B88002BA1
S31508008B4036D1A8E0144B188808B1FFF713FA114B71
S31508008B5093F82F3013F0010F0CD007236376002308
S31508008B60A3760120FFF706FA10220C4B1A70FBF7C2
S31508008B7023FF1DE0084B1B88D3B98CE0074B1B78F5
S31508008B8013F0010F00F08780072363760023A3768E
S31508008B9081E000BFA42A0020102A00201C2A0020F9
S31508008BA0242A0020901A0020E6300020142A0020EB
S31508008BB010223C4B83F82F2028223B4B1A80502248
S31508008BC0384B83F82E20227A364B83F82A20627A8D
S31508008BD083F82B20A27A83F82C20E27A83F82D20BA
S31508008BE0227B83F82620627B83F82720A27B83F8E2
S31508008BF02820E27B83F829200622DA75A2885A847F
S31508008C00E2889A84294A1188598352889A83228845
S31508008C10DA8362881A84637E13F0100F06D0214B1C
S31508008C20002283F8312083F8302006E01D4B062207
S31508008C3083F830200A2283F831201A4C4023A37582
S31508008C40194B1B881A0A22746374002384F835307A
S31508008C5084F8343084F8323084F83330FFF730FA49
S31508008C60C04360860F4C4523A3730022E2736275E6
S31508008C7022750F490B8801339BB20B80190AA17420
S31508008C80E37422766276FFF7EDF9C043208300226B
S31508008C90084B1A7070BD0023034A1380054A1370E7
S31508008CA070BD00BFA42A0020102A0020A02A002098
S31508008CB0921A00201C2A0020F8B505460E46254AB9
S31508008CC0138801339BB21380B3F5FA4F03D34FF4DD
S31508008CD08052204B1A8000221F4B1A700CE01F4B43
S31508008CE003EB84139F881B4B1888FFF7B5F9874257
S31508008CF0E5D00134184B1C70174B1C78002CEED0AD
S31508008D0000221A700BE0154A02EB831292881AB9F0
S31508008D10124800EB831007E001330F4A13700E4B1D
S31508008D201B78002BEFD0002088B10A4B1A88130A4B
S31508008D3043EA02238380C68015B90023036003E053
S31508008D402B8803806B88438040230372F8BD00207C
S31508008D50F8BD00BF981A00209A1A0020E8300020B3
S31508008D6000290CDD08B58AB2054B1A80054B1B682D
S31508008D70834203D00146184600F0F3FC08BD70474D
S31508008D80E6300020142A0020F0B400223B4B1A706B
S31508008D903B4E1EE03A4D5A001A4494002E192C5B9D
S31508008DA0A4B103EB4305AA00354D2A4452886AB19B
S31508008DB00588AC420AD14488A24207D10C6874607F
S31508008DC0898831812F4A1278B27254E001332B4ACE
S31508008DD013702A4B1B78072BDCD90022274B1A70F5
S31508008DE00FE0274D5A001A4494002E192A5B2AB917
S31508008DF003EB4304A2002A44528832B101331F4AC6
S31508008E0013701E4B1B78072BEBD9082B28D1002390
S31508008E101D4A13701D4A1370184A137013E0194A35
S31508008E20147803EB4305AA00154D2A44927AA61A2C
S31508008E30154D2D78AE4203DD134A1670134A13708A
S31508008E4001330E4A13700D4B1B78072BE7D90F4BCE
S31508008E501B780A4A137003EB43039A00084E16441C
S31508008E600268334643F8042B0A6872608A889A8037
S31508008E70044B1B78B372F0BC704700BFA21A0020DF
S31508008E80A41A0020051B0020A31A0020041B00209A
S31508008E9010B4154B1C780134E4B21C700022134B35
S31508008EA01A7019E012485A001A4491004218415A99
S31508008EB052880A430DD003EB43018A000244927A92
S31508008EC0A21A772A05DD03EB43018A000020084928
S31508008ED088500133054A1370044B1B78072BE1D9D8
S31508008EE05DF8044B704700BF051B0020A21A00203E
S31508008EF0A41A002010B5324B1B88292B03D8002250
S31508008F002F4B1A8010BD00222D4B1A802D4B9B8AA1
S31508008F10B3F5807F03D0B3F5007F3FD010BD294B52
S31508008F20DA8C294B1B889A4249D1264B1A8D264B37
S31508008F305B889A4243D1254C2146A01DFFF724FFA2
S31508008F40002204F8022C022204F8012C2168C4F835
S31508008F500A10A188E1811E49086820608988A180D5
S31508008F6044F8100C24F80C1CD4F80A1044F8161C03
S31508008F70E28924F8122CE288228222896282124A25
S31508008F801188E18052882281082204F80A2C0622D8
S31508008F9004F8092C2A220A4B1A8010BD094BDA8CD0
S31508008FA0094B1B889A420AD1064B1A8D064B5B88D9
S31508008FB09A4204D1054801460630FFF7E5FE10BD82
S31508008FC0102A0020A42A0020A02A0020BA2A00205D
S31508008FD09C1A002030B44C4BD98B8AB24FF6FF73DB
S31508008FE09A420CD1484B188C4FF6FF73984206D11B
S31508008FF0454B464A1068186092889A8073E0444B3D
S315080090001B88444800885340184209D13E4B1A8CA5
S3150800901094B23F4B5B883F4840886340184206D06D
S315080090203D4B3E4A1188198052885A8002E03A4BD5
S3150800903019805A8000223A4B1A703A4D16E0394880
S315080090405A001A4491004518334A1488425A9442E1
S3150800905009D1314A508803EB43018A0031490A4451
S315080090605288904206D001332D4A13702C4B1B7838
S31508009070072BE4D9082B30D1234B4FF0FF321A6067
S315080090809A8000221A629A8427490868C3F806005B
S3150800909089885981C3F8160059831F490888D884D6
S315080090A0498819851A49088898834988D9831A7579
S315080090B0012159759A73D973082119745A740622AD
S315080090C09A740422DA74197306225A733633174AC5
S315080090D013602A22164B1A8014E00B4B55F8042FFE
S315080090E01A60AA889A80084B0F4A1168C3F80610B6
S315080090F092885A8108221A7300225A730C4A1388D6
S315080091000E33138030BC7047A42A0020AC9F000899
S31508009110A02A00209C2A0020081B0020982A00204C
S31508009120A21A0020A41A00209C1A0020242A002033
S31508009130102A002010B504464160F9F7D7F92060D7
S3150800914010BD00BF10B50446F9F7D0F92368C01A58
S3150800915063689842B4BF0020012010BD3523037010
S315080091600123437081700330704700BF03463622DF
S31508009170027004224270034A1068C3F80200981D60
S31508009180704700BF281B0020372303700323437052
S3150800919001228270C370062303710530704700BF31
S315080091A0FF23037001307047074B828C1A80C28CEC
S315080091B05A80064B028D1A80428D5A80044B028EC5
S315080091C01A80428E5A807047A02A00209C2A0020C6
S315080091D0982A002003463222027004224270034A6B
S315080091E01068C3F80200981D704700BF301B0020A6
S315080091F010B40346014400242EE01A78332A24D0FA
S3150800920006D8032A10D0062A13D0012A21D106E04F
S31508009210362A15D0FF2A21D0352A1AD10EE0D3F8DE
S315080092200200104A906214E0D3F802000D4A106357
S315080092300FE0D3F802000B4AD0620AE09C7808E0F7
S31508009240D3F80200074AD06103E0D3F80200054AC2
S3150800925010625A78023213448B42CED320465DF808
S31508009260044B70470C1B0020F8B504460123037015
S315080092704370194B9A6982700025C570174A1068A1
S315080092806060258180276781154A1268E26025613A
S315080092906561A5619E693246596904F11C0000F0B2
S315080092A060FA06F118002044C6F110022946043077
S315080092B000F062FA4022294604F12C0000F05CFA1C
S315080092C03A46294604F16C0000F056FA054B186830
S315080092D0C4F8EC00F8BD00BF0C1B0020B49F0008C2
S315080092E0A02A0020B89F000838B50A4C25682846E9
S315080092F0FFF7BAFF012105F1F000FFF72FFFFFF78F
S3150800930043FFFFF74DFF2368C11A1846FFF728FDEC
S3150800931038BD00BF242A002038B50B4C25682846DE
S31508009320FFF7A2FF032105F1F000FFF717FFFFF78C
S315080093301DFFFFF74FFFFFF733FF2368C11A1846D3
S31508009340FFF70EFD38BD00BF242A002010B5114BCB
S315080093501C682378022B17D104220F49A01800F0A5
S31508009360F1F998B90D4B9A69596904F11C0000F096
S31508009370E9F968B92069094B5862094B198804F15B
S31508009380F000FFF735FF10BD002010BD002010BD0E
S31508009390002010BD242A0020B49F00080C1B0020C2
S315080093A0102A002010B582B00C4C6061A161002320
S315080093B0A3704FF6FF73ADF80430ADF806304FF4DE
S315080093C0864101A8FFF778FC606010B14FF4884326
S315080093D083800022014B1A8002B010BD0C1B0020AE
S315080093E0024B00221A805A80704700BFA02A00202C
S315080093F038B59E4B1B88B3F5937F7FD010D840F2C3
S315080094000F12934234D0B3F5887F01D2EBB118E13D
S31508009410B3F5887F34D040F22512934266D010E126
S31508009420B3F5AB7F00F0BF8005D840F255129342E2
S3150800943000F0B28005E1B3F5B57F00F0CE8040F2CA
S315080094406B12934200F0D080FBE0884B01229A70A1
S315080094504FF47A721A61FFF747FF844C216904F1C9
S315080094600800FFF767FE40F20F132380002300E091
S315080094700123002B00F0EA804FF488727B4B1A8098
S315080094807B4B1B7813F0020F05D17A48FFF75AFE7B
S31508009490002800F0DD80764B1B7813F0020F07D00A
S315080094A0FFF754FF022803D10222704B9A700CE092
S315080094B06E4B1B694EF65F22934202DC5B006B4AD9
S315080094C013616A4B9B78022BC5D14FF47A72674BAE
S315080094D01A61FFF721FF654C216904F10800FFF7BF
S315080094E029FE40F225132380002300E00123002BE8
S315080094F000F0B0804FF493725C4B1A805C4B1B787B
S3150800950013F0020F05D15B48FFF71CFE002800F098
S31508009510A380574B1B7813F0020F07D0FFF716FFEF
S31508009520052803D10322514B9A7011E04F4B1B6952
S3150800953042F21072934207DC4C4A03F57A731361C0
S315080095409378032BC5D103E00020484B188038BD1B
S315080095504648FFF729FE454D288CFEF77DFD040495
S31508009560688CFEF779FD204340084FF47A7303FBB5
S3150800957000F0002801DB286103E06FF000423B4B56
S315080095801A613A4C216904F10800FFF7D3FD40F24D
S3150800959055132380002300E00123002B5ED04FF4EF
S315080095A0AB72324B1A803348FFF7CCFD002857D0F0
S315080095B02E4B02229A704FF47A721A61FFF710FF47
S315080095C0FFF7AAFE294C216904F10800FFF7B2FD4E
S315080095D04FF4B5732380002300E00123002B41D00C
S315080095E040F26B12214B1A80214B1B7813F0020FA5
S315080095F004D12048FFF7A6FD002835D01C4B1B7860
S3150800960013F0020F07D0FFF7A1FE052803D10322A6
S31508009610164B9A7011E0154B1B6942F21072934271
S3150800962007DC124A03F57A7313619378032BC7D1C3
S3150800963003E000200D4B188038BD0C48FFF7B4FD39
S3150800964089E70022094B1A80022038BD032038BD5D
S31508009650002038BD032038BD002038BD032038BDA2
S31508009660002038BD032038BD002038BD0C1B002063
S315080096701C2A0020141B002008B5FFF7B9FE08BDF8
S3150800968008B5074B044613B10021AFF30080054B1C
S315080096901868836A03B198472046F9F797FA00BF16
S315080096A000000000BC9F000870B50E4B0E4CE41A73
S315080096B0A41000251E46A54204D056F82530984722
S315080096C00135F8E700F06EF8084C094BE41AA410C7
S315080096D000251E46A54204D056F825309847013580
S315080096E0F8E770BDF4020020F4020020F80200201A
S315080096F0F4020020034B1B68186A034B002808BFB6
S3150800970018467047840100208801002008B5034BDD
S315080097101868FFF7EFFFD0F8EC0008BD84010020B9
S3150800972082B001B901A93AB143B113780B60127836
S31508009730101C18BF012003E0104601E06FF001007D
S3150800974002B0704710B501390244904207D010F8AC
S31508009750013B11F8014FA342F7D0181B10BD00209A
S3150800976010BD10B5431E0A44914204D011F8014BAE
S3150800977003F8014FF8E710BD02440346934202D0AE
S3150800978003F8011BFAE7704749B1FF2A85BF8A2308
S3150800979003600A704FF0FF3098BF012070470846F3
S315080097A070470000F8B500BFF8BC08BC9E46704775
S315080097B0F8B500BFF8BC08BC9E46704757696E5599
S315080097C053422042756C6B204465766963650000D8
S315080097D04F70656E424C5420557365720000000048
S315080097E03030303030303030303530430000000013
S315080097F044656661756C740057696E55534220421C
S31508009800756C6B20496E746572666163650000004D
S315080098106C69622F7569702F6E65746465762E6340
S31508009820000000002F64656D6F70726F675F6F6C64
S31508009830696D65785F73746D3332653430372E73AE
S31508009840726563002F626F6F746C6F672E7478741D
S31508009850000000004F70656E424C5400303A00001C
S315080098602E2E2F2E2E2F2E2E2F536F757263652FA9
S3150800987066696C652E6300004669726D776172656C
S3150800988020757064617465207265717565737420DE
S3150800989064657465637465640A0D00004F70656ECF
S315080098A0696E67206669726D776172652066696C94
S315080098B06520666F722072656164696E672E2E2E4A
S315080098C0000000004552524F520A0D004F4B0A0D38
S315080098D0000000005374617274696E6720746865CD
S315080098E02070726F6772616D6D696E67207365713E
S315080098F075656E63650A0D0050617273696E67203F
S315080099006669726D776172652066696C6520746F29
S315080099102064657465637420657261736520626C82
S315080099206F636B732E2E2E0045726173696E672006
S31508009930000000002062797465732066726F6D20DE
S315080099406D656D6F727920617420307800000000B3
S3150800995052656164696E67206C696E652066726F10
S315080099606D2066696C652E2E2E4552524F520A0D91
S3150800997000000000496E76616C696420636865635F
S315080099806B73756D20666F756E642E2E2E4552525A
S315080099904F520A0D0000000050726F6772616D6DBC
S315080099A0696E672000000000206279746573207470
S315080099B06F206D656D6F72792061742030780000B4
S315080099C057726974696E672070726F6772616D206D
S315080099D0636865636B73756D2E2E2E00436C6F730B
S315080099E0696E67206669726D776172652066696C53
S315080099F0650A0D004669726D776172652075706437
S31508009A00617465207375636365737366756C6C79C9
S31508009A1020636F6D706C657465640A0D0000000044
S31508009A202E2E2F2E2E2F2E2E2F536F757263652FE7
S31508009A3041524D434D345F53544D333246342F759E
S31508009A4073622E63000000002E2E2F2E2E2F2E2E30
S31508009A502F536F757263652F41524D434D345F53D3
S31508009A60544D333246342F756172742E63000000EC
S31508009A7000000800100018002000280030003800F8
S31508009A804000480050005800800088009000980068
S31508009A90A000A800B000B800C000C800D000D800D8
S31508009AA000C0000800400000030000000000010894
S31508009AB00000010004000000000002080000020087
S31508009AC0050000000000040800000200060000006F
S31508009AD00000060800000200070000000000080851
S31508009AE0000002000800000000000A08000002004A
S31508009AF00900000000000C08000002000A0000002F
S31508009B0000000E08000002000B0000002E2E2F2E6B
S31508009B102E2F2E2E2F536F757263652F41524D438C
S31508009B204D345F53544D333246342F63616E2E6382
S31508009B3000000000050206020603070308030903DE
S31508009B4009040A040B040C040C050D050E050F0583
S31508009B500F06100610071008222A3A3C3E3F7C7F63
S31508009B60000000002B2C3B3D5B5D0000809A4541C0
S31508009B708E418F804545454949498E8F9092924F2F
S31508009B80994F555559999A9B9C9D9E9F41494F556A
S31508009B90A5A5A6A7A8A9AAABACADAEAFB0B1B2B3FE
S31508009BA0B4B5B6B7B8B9BABBBCBDBEBFC0C1C2C3EF
S31508009BB0C4C5C6C7C8C9CACBCCCDCECFD0D1D2D3DF
S31508009BC0D4D5D6D7D8D9DADBDCDDDEDFE0E1E2E3CF
S31508009BD0E4E5E6E7E8E9EAEBECEDEEEFF0F1F2F3BF
S31508009BE0F4F5F6F7F8F9FAFBFCFDFEFF01030507A5
S31508009BF0090E10121416181C1E0000007D1D010007
S31508009C00632C001E9601A01E5A01001F0806101F8D
S31508009C100606201F0806301F0806401F0606511FA5
S31508009C200700591F521F5B1F541F5D1F561F5F1FDA
S31508009C30601F0806701F0E00BA1FBB1FC81FC91F6A
S31508009C40CA1FCB1FDA1FDB1FF81FF91FEA1FEB1FFE
S31508009C50FA1FFB1F801F0806901F0806A01F08068C
S31508009C60B01F0400B81FB91FB21FBC1FCC1F0100CC
S31508009C70C31FD01F0206E01F0206E51F0100EC1FE6
S31508009C80F21F0100FC1F4E21010032217021100233
S31508009C90842101008321D0241A05302C2F04602C3E
S31508009CA00201672C0601752C0201802C6401002D27
S31508009CB0260841FF1A03000061001A03E000170393
S31508009CC0F8000703FF0001007801000130013201A6
S31508009CD00601390110014A012E01790106018001A8
S31508009CE04D004302810182018201840184018601BB
S31508009CF08701870189018A018B018B018D018E01FC
S31508009D008F0190019101910193019401F601960149
S31508009D109701980198013D029B019C019D01200233
S31508009D209F01A001A001A201A201A401A401A6010C
S31508009D30A701A701A901AA01AB01AC01AC01AE01BB
S31508009D40AF01AF01B101B201B301B301B501B5016C
S31508009D50B701B801B801BA01BB01BC01BC01BE011B
S31508009D60F701C001C101C201C301C401C501C40193
S31508009D70C701C801C701CA01CB01CA01CD0110013B
S31508009D80DD0101008E01DE011201F3010300F1017C
S31508009D90F401F401F8012801220212013A0209002D
S31508009DA0652C3B023B023D02662C3F024002410203
S31508009DB0410246020A01530240008101860155020A
S31508009DC089018A0158028F015A0290015C025D02DC
S31508009DD05E025F02930161026202940164026502F7
S31508009DE066026702970196016A02622C6C026D028E
S31508009DF06E029C01700271029D01730274029F013A
S31508009E0076027702780279027A027B027C02642C57
S31508009E107E027F02A60181028202A90184028502CE
S31508009E2086028702AE014402B101B20145028D02E3
S31508009E308E028F0290029102B7017B030300FD0395
S31508009E40FE03FF03AC0304008603880389038A0321
S31508009E50B1031103C2030200A303A303C403080347
S31508009E60CC0303008C038E038F03D8031801F20377
S31508009E700A00F903F303F403F503F603F703F703FC
S31508009E80F903FA03FA0330042003500410076004A8
S31508009E9022018A043601C1040E01CF040100C00460
S31508009EA0D00444016105260400000000C700FC0038
S31508009EB0E900E200E400E000E500E700EA00EB0064
S31508009EC0E800EF00EE00EC00C400C500C900E6009B
S31508009ED0C600F400F600F200FB00F900FF00D60009
S31508009EE0DC00A200A300A500A7209201E100ED0076
S31508009EF0F300FA00F100D100AA00BA00BF0010234F
S31508009F00AC00BD00BC00A100AB00BB0091259225AA
S31508009F109325022524256125622556255525632581
S31508009F20512557255D255C255B25102514253425E7
S31508009F302C251C2500253C255E255F255A255425FC
S31508009F4069256625602550256C25672568256425BD
S31508009F50652559255825522553256B256A25182523
S31508009F600C25882584258C2590258025B103DF00BE
S31508009F709303C003A303C303B500C403A60398034E
S31508009F80A903B4031E22C603B50329226122B10020
S31508009F906522642220232123F7004822B0001922D3
S31508009FA0B7001A227F20B200A025A000FFFFFFFFFE
S31508009FB0FFFF0000ADDE12236382536324010020F5
S31508009FC04300504F534958002E00002020202020DF
S31508009FD0202020202828282828202020202020204B
S31508009FE0202020202020202020202088101010103B
S31508009FF0101010101010101010101004040404048F
S3150800A00004040404041010101010101041414141BA
S3150800A01041410101010101010101010101010101A2
S3150800A02001010101010110101010101042424242B4
S3150800A0304242020202020202020202020202020272
S3150800A0400202020202021010101020000000000096
S3150800A05000000000000000000000000000000000F2
S3150800A06000000000000000000000000000000000E2
S3150800A07000000000000000000000000000000000D2
S3150800A08000000000000000000000000000000000C2
S3150800A09000000000000000000000000000000000B2
S3150800A0A000000000000000000000000000000000A2
S3150800A0B00000000000000000000000000000000092
S3150800A0C00000000000000000000000000000000082
S30D0800A0D01461FF7F0100000086
S3150800A0D8690300086D030008710300087503000882
S3150800A0E87D03000885030008910300089D030008FE
S3150800A0F8A9030008D1030008B5030008ED03000802
S3150800A10809040008250400080403090412011001BB
S3150800A11800000040501DAC60000101020301000068
S3150800A128F1040008D90400087904000800000000B2
S3150800A13800000000610400086D0400084D040008CA
S3150800A1480000000000000000410400080902200081
S3150800A158010100C0320904000002FF0000000705DB
S3150800A16881024000FF070501024000FFE0000020C9
S3150800A178212100086D2000081D200008851F0008F9
S3150800A188ED1F0008691F0008511F0008951F0008E1
S3150800A198A51F0008B51F0008CD1F0008000000000D
S3150800A1A80102030401020304060708090100000066
S3150800A1B80101040000000000000000000000000083
S3150800A1C80000000000000000000000000000000079
S3150800A1D80000000000000000000000000000000069
S3150800A1E80000000000000000000000000000000059
S3150800A1F80000000000000000000000000000000049
S3150800A2080000000000000000000000000000000038
S3150800A21800000000240100204300000000000000A0
S3150800A2280000000000000000000000000000000018
S3150800A23800000000000000004300000000000000C5
S3150800A24800000000000000000000000000000000F8
S3150800A25800000000000000004300000000000000A5
S3150800A26800000000000000000000000000000000D8
S3150800A2780000000000000000430000000000000085
S3150800A28800000000000000000000000000000000B8
S3150800A2980000000000000000430000000000000065
S3150800A2A80000000000000000000000000000000098
S3150800A2B80000000000000000430000000000000045
S3150800A2C80000000000000000000000000000000078
S3150800A2D80000000000000000430000000000000025
S3150800A2E80000000000000000000000000000000058
S3150800A2F80000000000000000899700082197000860
S3150800A30800000000CA9F0008C89F0008C99F0008E7
S3150800A318C99F0008C99F0008C99F0008C99F000867
S3150800A328C99F0008C99F0008C99F0008C99F000857
S3150800A338FFFFFFFFFFFFFFFFFFFFFFFFFFFF000015
S3150800A348010041534349490000000000000000008D
S3150800A35800000000000000000000000000000000E7
S3150800A368000041534349490000000000000000006E
S3150800A37800000000000000000000000000000000C7
S3110800A38800000000AD0100088901000873
S70508000000F2
